:020000040800F2
:10000000300D0020210300081D0300081D03000817
:100010001D0300081D0300081D0300080000000068
:100020000000000000000000000000001D030008A8
:100030001D030008000000001D0300081D03000848
:100040001D0300081D0300081D0300081D03000810
:100050001D0300081D0300081D0300081D03000800
:100060001D0300081D0300081D0300081D030008F0
:100070001D0300081D0300081D0300081D030008E0
:100080001D0300081D0300081D03000800000000F8
:100090000000000000000000000000001D03000838
:1000A0001D0300081D0300081D0300081D030008B0
:1000B000B1200008F50100081D0300081D03000819
:1000C0001D0300081D0300081D0300081D03000890
:1000D0001D0300083D2000081D03000875200008CE
:1000E0001D0300081D0300081D0300080000000098
:1000F0000000000000000000000000000000000000
:1001000000000000000000000000000000000000EF
:1001100000000000000000001D0300081D0300088F
:100120005FF808F130B5012185B01A4D022003F0C7
:1001300037FB0021022003F04FFB00240523284653
:1001400001A9ADF80430ADF80640ADF80840ADF8AF
:100150000A408DF80C4000F05FF82846012100F0BD
:10016000D9F801221146284600F0C2F801231D22C9
:1001700068468DF800208DF802308DF803308DF838
:10018000014003F02BFF2146284600F099F805B006
:1001900030BD00BF0004004010B5044600210D48EA
:1001A00000F08EF821460B4800F0A6F8002109481F
:1001B00000F0A0F80121074800F082F8064A002369
:1001C00013701378002BFCD000210248BDE81040CA
:1001D00000F076B8000400403006002048B110B5A9
:1001E000044600214FF47A70FFF7D6FF013CF8D1A6
:1001F00010BD704708B50121054800F07FF830B107
:100200000121034800F086F8024B01221A7008BD54
:100210000004004030060020264A038890429BB22A
:1002200012D002F5006290420ED0B0F1804F0BD098
:10023000A2F59832904207D002F58062904203D036
:1002400002F58062904203D14A8823F07003134381
:10025000194A904226D002F58062904222D0CA8884
:1002600070B423F44073134C8E880D889BB21343F3
:10027000A0420380868505850ED0104B98420BD096
:1002800003F54063984207D003F58063984203D09A
:1002900003F58063984201D10B7A038601238382A0
:1002A00070BC704703808B8883850B88038501238E
:1002B00083827047002C0140001000400034014050
:1002C000038829B923F001031B041B0C038070472A
:1002D0009BB243F001030380704700BF83899BB248
:1002E0001AB923EA0101818170471943818170475E
:1002F000FFF7F4BF8184704781857047038A828944
:1003000011EA030092B203D0114214BF0120002071
:10031000704700BFC94389B201827047FEE700BF42
:100320000E4A0F4B9A420DD2D0430E4918440B4649
:1003300020F003000430084453F8041B834242F8C1
:10034000041BF9D1084809494FF000028842B8BFA0
:1003500040F8042BFADB02F0B1B900BF0000002026
:10036000F402002050A10008F4020020300900200F
:1003700010B504464021084803F034FC0028F9D0A9
:100380002146054803F026FC4021034803F02AFCDF
:100390000028F9D010BD00BF0048004038B5054620
:1003A000007838B100240134A4B2FFF7E1FF285DE2
:1003B0000028F8D138BD00BF38B51A4B00220A28F2
:1003C0001A7017D00546184C94F8C830E054FFF75F
:1003D000CFFF082D94F8C83004D13BB1013B84F81D
:1003E000C83038BDC52B0AD80D2D08D0013384F88C
:1003F000C83038BD0C4C94F8C830C52B11D90A2030
:10040000FFF7B6FF94F8C830002523440649074893
:100410005D7006F00FF9064B012284F8C8501A707F
:1004200038BD38BDB0070020F4020020B40600201B
:100430009D07002070B51A4904461A4806F0DAF8FC
:1004400058B9194D04464F200134A4B2FFF790FF6C
:10045000285D0028F8D1012070BD1449114806F02C
:10046000C9F850B9104D04464F200134A4B2FFF72B
:100470007FFF285D0028F8D170BD0D49094806F0BE
:10048000B9F80028EED00B4E00254F200135ADB253
:10049000FFF76EFF705D0028F8D1204670BD00BFE9
:1004A000389A000834060020FC8B00083C990008AC
:1004B000088C00080C8C0008012838B50AD00B4DB8
:1004C00000244F200134A4B2FFF752FF285D00281A
:1004D000F8D138BD064D00244F200134A4B2FFF7F7
:1004E00047FF285D0028F8D138BD00BF348C0008D4
:1004F0002C8C00082DE9F04F1C481D4903781D4C39
:100500000022202B89B00A70227000F08086002B18
:1005100000F091850D2B00F07E8605460DF103015C
:1005200001F8013F15F8013F0132202B00F0A185B1
:10053000002B00F081850D2B00F0A285182AEFD149
:10054000037E0021202B8DF81C1005D1811811F895
:10055000013F0132202BFAD0002B00F06B860D2BCF
:1005600000F09385044D024400210BE0B406002006
:100570009D07002090070020330600200D2B08D097
:10058000772906D005F8013F12F8013F0131002B11
:10059000F4D1A94B00225A5401A8A84906F02AF820
:1005A000002800F04783A64901A806F023F8002898
:1005B00000F04083A34901A806F01CF8002840F091
:1005C0004285A14E05460A200135ADB2FFF7D0FEA7
:1005D000705D0028F8D19D4E05464220FFF7C8FE09
:1005E000681C85B2705D0028F8D1994E05463078B8
:1005F000FFF762FFDFF894824C273846FFF7B8FE1A
:10060000681C85B218F80570002FF6D1914B8A4D01
:100610001878FFF751FF96F8D0308F4A03F00703A0
:1006200052F8232028468D4905F0C0FF287830B1C4
:100630000137BFB2FFF79CFEE85D0028F8D1D6F87D
:10064000D430642202FB03F285497B4805F0AEFFFB
:100650002878002730B10137BFB2FFF789FEE85D87
:100660000028F8D173687F4A7F49A2FB03327248A1
:10067000920905F09BFF2878002730B10137BFB2FF
:10068000FFF776FEE85D0028F8D1DFF804924FF01E
:100690000008522708F1010838461FFA88F8FFF7CA
:1006A00067FE19F80870002FF4D1B078FFF704FF47
:1006B000D6F8CC80404604F079FF814604F05CFD1A
:1006C0000146404604F0A2FC684904F0A9FD04F08C
:1006D0006DFF4A4603466649574805F067FF28788C
:1006E00030B10137BFB2FFF743FEE85D0028F8D113
:1006F000604A6149504805F059FF2878002730B119
:100700000137BFB2FFF734FEE85D0028F8D1B268C8
:100710005A49494805F04AFF2878002730B1013787
:10072000BFB2FFF725FEE85D0028F8D1337B4FF418
:10073000877202FB03F252493F4805F037FF2878E1
:10074000002730B10137BFB2FFF712FEE85D002885
:10075000F8D1727B4B49384805F028FF28780027EC
:1007600030B10137BFB2FFF703FEE85D0028F8D1D2
:10077000B27B4549304805F019FF2878002730B191
:100780000137BFB2FFF7F4FDE85D0028F8D1DFF8CC
:1007900004810027522301371846BFB2FFF7E8FD56
:1007A00018F80730002BF6D1F07BDFF8EC801F46FD
:1007B000FFF782FE52231846FFF7DAFD7B1C9FB23B
:1007C00018F80730002BF6D1B07CDFF8D0801F4638
:1007D000FFF772FE52231846FFF7CAFD7B1C9FB23B
:1007E00018F80730002BF6D1307CDFF8B4801F46B4
:1007F000FFF762FE52231846FFF7BAFD7B1C9FB23B
:1008000018F80730002BF6D1707CDFF898801F466F
:10081000FFF752FE5220FFF7ABFD7B1C9FB218F88A
:1008200007000028F7D10746DFF87C80F07CFFF74F
:1008300043FE52203AE000BF340600203C8C000802
:10084000448C0008D0940008D8940008F494000860
:1008500004000020AC060020DC8B00080495000892
:100860001C950008D34D62102C95000800007A44B6
:1008700044950008980000206C95000880950008B9
:1008800098950008AC950008C4950008FC940008F1
:100890003C950008DC950008F095000800960008DB
:1008A000109600082096000838960008FFF760FDB3
:1008B000781C87B218F807000028F7D1707DFFF781
:1008C000FBFDF27D002A00F0EA835200AE49AF48FA
:1008D00005F06CFE2878002730B10137BFB2FFF772
:1008E00047FDE85D0028F8D1DFF8F08200275223A9
:1008F00001371846BFB2FFF73BFD18F80730002B51
:10090000F6D1B07D9846FFF7D7FDDFF8D4924127A6
:100910003846FFF72DFD08F101031FFA83F819F897
:100920000870002FF4D1307EFFF7C6FDD6F8C880DE
:10093000404604F03BFE814604F01EFC0146404662
:1009400004F064FB924904F06BFC04F02FFE4A466D
:10095000034690498D4805F029FE287830B10137CB
:10096000BFB2FFF705FDE85D0028F8D18A4A8B4940
:10097000D01D12F8013F202B08BF0023824201F84E
:10098000013FF6D196F8C730854A86497F4805F081
:100990000DFE2878002730B10137BFB2FFF7E8FC21
:1009A000E85D0028F8D1804A8049784805F0FEFDCE
:1009B0002878002730B10137BFB2FFF7D9FCE85DD6
:1009C0000028F8D17A4A7B49704805F0EFFD287875
:1009D000002730B10137BFB2FFF7CAFCE85D00283D
:1009E000F8D1727E7449694805F0E0FD2878002747
:1009F00030B10137BFB2FFF7BBFCE85D0028F8D18A
:100A0000DFF8E0914FF00008412708F1010838466F
:100A10001FFA88F8FFF7ACFC19F80870002FF4D122
:100A2000307FFFF749FDB27F6449584805F0BEFDAD
:100A3000287830B10137BFB2FFF79AFCE85D002893
:100A4000F8D15F4A5F49514805F0B0FD287800278A
:100A500030B10137BFB2FFF78BFCE85D0028F8D159
:100A6000DFF884810027412301371846BFB2FFF722
:100A70007FFC18F80730002BF6D1707FDFF86C810F
:100A80001F46FFF719FD41231846FFF771FC7B1C39
:100A90009FB218F80730002BF6D196F8FA00DFF86D
:100AA00050811F46FFF708FD4320FFF761FC7B1CC8
:100AB0009FB218F807000028F7D10746DFF8348105
:100AC00096F88500FFF7F8FC43231846FFF750FC23
:100AD000781C87B218F80730002BF6D196F8A400DE
:100AE00050B11F46DFF81081FFF742FC7B1C9FB21C
:100AF00018F807000028F7D196F8862032492348D5
:100B000005F054FD2878002730B10137BFB2FFF758
:100B10002FFCE85D0028F8D196F887202B491B4868
:100B200005F044FD2878002730B10137BFB2FFF748
:100B30001FFCE85D0028F8D196F88320002A00F019
:100B4000A78252002249114805F030FD287800277D
:100B500030B10137BFB2FFF70BFCE85D0028F8D1D8
:100B60001C4F0025432301351846ADB2FFF700FCAA
:100B70007B5D002BF7D196F88900174F1D46FFF7D4
:100B80009BFC43203AE000BF4C960008340600204E
:100B900000007A448C9600088D0000207B0700201E
:100BA0007C070020AC960008E0000020C4960008F6
:100BB000C6000020D8960008EC9600080C970008A4
:100BC00023000020289700087097000888970008E5
:100BD0009C970008C8970008D497000878960008EA
:100BE0008496000800970008409700084C9700087A
:100BF0005897000860970008A8000020FFF7B8FB8E
:100C00006B1C9DB2785D0028F8D1054696F88800E7
:100C1000074EFFF751FC6320FFF7AAFB681C85B263
:100C2000705D0028F8D1207809B0BDE8F08F00BFD2
:100C3000A09C0008A64E05460A200135ADB2FFF77C
:100C400097FB705D0028F8D1A24E05464220FFF7C1
:100C50008FFB681C85B2705D0028F8D19E4E05465A
:100C60004C20FFF785FB681C85B2705D0028F8D129
:100C70009A4E05465020FFF77BFB681C85B2705DDD
:100C80000028F8D1964E05464820FFF771FB681CF6
:100C900085B2705D0028F8D1924E05465320FFF7CB
:100CA00067FB681C85B2705D0028F8D18E4E054642
:100CB0005220FFF75DFB681C85B2705D0028F8D1FB
:100CC0008A4E05465220FFF753FB681C85B2705DC3
:100CD0000028F8D1864E05465220FFF749FB681CD4
:100CE00085B2705D0028F8D1824E05464220FFF79C
:100CF0003FFB681C85B2705D0028F8D17E4E05462A
:100D00004420FFF735FB681C85B2705D0028F8D1E0
:100D10007A4E05465320FFF72BFB681C85B2705DA9
:100D20000028F8D1764E05465320FFF721FB681CBA
:100D300085B2705D0028F8D1724E05465420FFF749
:100D400017FB681C85B2705D0028F8D16E4E054611
:100D50004120FFF70DFB681C85B2705D0028F8D1BB
:100D60006A4E05465320FFF703FB681C85B2705D91
:100D70000028F8D1664E05464320FFF7F9FA681CB3
:100D800085B2705D0028F8D1624E05465520FFF708
:100D9000EFFA681C85B2705D0028F8D15E4E0546FA
:100DA0005220FFF7E5FA681C85B2705D0028F8D183
:100DB0005A4E05465220FFF7DBFA681C85B2705D7B
:100DC0000028F8D1564E05465320FFF7D1FA681C8B
:100DD00085B2705D0028F8D1524E05464120FFF7DC
:100DE000C7FA681C85B2705D0028F8D14E4E0546E2
:100DF0004120FFF7BDFA681C85B2705D0028F8D16C
:100E00004A4E05464120FFF7B3FA681C85B2705D73
:100E10000028F8D1464E05465320FFF7A9FA681C72
:100E200085B2705D0028F8D1424E05464120FFF79B
:100E30009FFA681C85B2705D0028F8D13E4E0546C9
:100E40005320FFF795FA681C85B2705D0028F8D131
:100E50003A4E05465220FFF78BFA681C85B2705D4A
:100E60000028F8D1364E05464120FFF781FA681C6C
:100E700085B2705D0028F8D1324E05465420FFF748
:100E800077FA681C85B2705D0028F8D12E4E0546B1
:100E90005420FFF76DFA681C85B2705D0028F8D108
:100EA0002A4E05464120FFF763FA681C85B2705D43
:100EB0000028F8D1264E05464120FFF759FA681C54
:100EC00085B2705D0028F8D1224E0546432043E0EC
:100ED000488C0008788C0008A48C0008C08C00089E
:100EE000EC8C0008288D00086C8D0008908D00089F
:100EF000C88D0008008E0008288E0008508E00085B
:100F0000788E0008A88E0008EC8E0008288F000854
:100F1000588F0008888F0008C08F000810900008C4
:100F20004090000888900008AC900008D890000815
:100F3000109100083491000864910008A491000801
:100F4000D4910008109200085C920008909200086A
:100F5000C892000808930008FFF70AFA681C85B2D7
:100F6000705D0028F8D1B54E05464320FFF700FA22
:100F7000681C85B2705D0028F8D1B14E054643204B
:100F8000FFF7F6F9681C85B2705D0028F8D1AD4E08
:100F900005464320FFF7ECF9681C85B2705D002818
:100FA000F8D1A94E05464320FFF7E2F9681C85B247
:100FB000705D0028F8D1A54E05464320FFF7D8F90B
:100FC000681C85B2705D0028F8D1A14E054643200B
:100FD000FFF7CEF9681C85B2705D0028F8D19D4EF0
:100FE00005464420FFF7C4F9681C85B2705D0028EF
:100FF000F8D1994E05464420FFF7BAF9681C85B22E
:10100000705D0028F8D1954E05465320FFF7B0F9E2
:10101000681C85B2705D0028F8D1914E05466320AA
:10102000FFF7A6F9681C85B2705D0028F8D120781A
:1010300009B0BDE8F08F1A4608AB1A44002302F845
:101040001C3CFFF7A9BA874901A805F0D3FA054669
:1010500060BB854805F0F6FA632840F2C980834EEC
:1010600054200135ADB2FFF783F9705D0028F8D147
:10107000D9E508AB0021134403F81C1CFFF766BA3E
:1010800008AB1A44002302F81C3C0021FFF781BA88
:10109000774F0FCF28606960AA60EB6056E5754F07
:1010A0000FCF28606960AA60EB6013E4724901A861
:1010B00005F0A0FA0546002871D0704901A805F096
:1010C00099FA0646002840F0E980674D284605F069
:1010D000B9FA092800F247816F1E0FE0D3B23B70C6
:1010E000A3F130022A2A6048A3F13A0300F22882D1
:1010F000062B40F2258205F0A5FA0136864280F0E3
:101100001D8217F8013FA3F161011929A3F1200203
:10111000E4D92D2BE4D10023AB5535446B78002B5B
:1011200000F02C81AA7803F00F03554E42B103EB77
:10113000830302F00F0202EB4303DBB20F2B01D853
:1011400086F8C730484805F07DFADFF81C814D4F1E
:10115000002506E018F8013B013507F8013F05F0CE
:1011600071FA85424048F5D3052D08D805F18A0368
:1011700045493344202203F8012B8B42FBD1002345
:101180001D460122414F86F8903022704F200135D4
:10119000ADB2FFF7EDF8785D0028F8D143E53248AD
:1011A00005F050FA0F283BD8394F3A4E0DE016F8AB
:1011B000013F0135A3F16102192A02D8203BDBB2BD
:1011C000337007F8013F05F03DFA85422648EED31B
:1011D00000231E462A4A2D4F154485F894304F208F
:1011E0000136B6B2FFF7C4F8B85D0028F8D11AE5A9
:1011F000421C1D492848254F05F0C4F94F200135F0
:10120000ADB2FFF7B5F8785D0028F8D10BE58DF8A1
:101210000420FFF79BB98DF804201146FFF7B9B9F8
:10122000124E54200135ADB2FFF7A2F8705D0028D0
:10123000F8D1F8E41946FFF7ACB900BF2C930008C9
:101240006493000890930008C49300081494000865
:10125000509400087494000890940008AC9400081E
:10126000A09C0008E097000834060020E8970008DA
:10127000B8970008689600080498000810980008BD
:10128000040000208D00002094000020FC8B00084A
:10129000970000203306002023000020B04901A859
:1012A00005F0A8F9054648BBAE4805F0CBF919286A
:1012B00000F2F980AC4FAD4E0DE016F8013F01355C
:1012C000A3F16102192A02D8203BDBB2337007F880
:1012D000013F05F0B7F98542A248EED300231E4630
:1012E000A34AA44F154485F8A4304F200136B6B266
:1012F000FFF73EF8B85D0028F8D194E49E4901A8B4
:1013000005F078F90546002844D1964805F09AF989
:10131000192835D8954E374608E02F2B13D82C2B9B
:1013200040F071818F4805F08DF90135854280F0DC
:10133000138117F8013FA3F161011929A3F12002DC
:10134000EBD8D3B23B70A3F13A02062A00F2A78091
:101350008A4E00254F200135ADB2FFF709F8705DC8
:101360000028F8D15FE43546854E54200135ADB2F2
:10137000FEF7FEFF705D0028F8D154E47C4EE1E6F4
:101380007F4E54200135ADB2FEF7F2FF705D0028AC
:10139000F8D148E47B4901A805F02CF9002800F0B9
:1013A0008D80794901A805F025F9002800F04B85CA
:1013B000764901A805F01EF90546002800F02D85A4
:1013C000734901A805F016F90546002800F0F984D4
:1013D000704901A805F00EF90546002800F0D484F4
:1013E0006D4901A805F006F90546002800F0A08423
:1013F0006A4901A805F0FEF80546002800F084843B
:10140000674901A805F0F6F80546002800F0508469
:10141000644901A805F0EEF80546002800F036847E
:10142000614901A805F0E6F8002800F0AF825F49A5
:1014300001A805F0DFF8002800F091825C4901A8BE
:1014400005F0D8F8002800F0D6825A4901A805F026
:10145000D1F8002840F0DB80424D2A782F2A05D0B1
:101460005C2A03D0A2F13003092B39D86B78202BEA
:1014700036D97E2B34D83E4900203E4F054681F8B0
:10148000C40081F8C22081F8C3304F200135ADB2CD
:10149000FEF76EFF785D0028F8D1FFF7C4BB5A2B2A
:1014A0003FF656AF3EE7364E54200135ADB2FEF75B
:1014B0005FFF705D0028F8D1FFF7B5BB294805F044
:1014C00030F8C3B2072B17D93B4E00253020013529
:1014D000ADB2FEF74DFF705D0028F8D1FFF7A3BB5A
:1014E000364E002543200135ADB2FEF741FF705D59
:1014F0000028F8D1FFF797BB1D4D194601226D203A
:1015000085F8D03002F09CF995F8D0302C4A154D72
:1015100003F0070352F8232028462A4905F046F82D
:10152000287800283FF47FAB00260136B6B2FEF7DC
:101530001FFFA85D0028F8D1FFF775BB0C4E04E62D
:101540000E4E00254F200135ADB2FEF711FF705D44
:101550000028F8D1FFF767BB1B4F00253DE000BF17
:101560004898000834060020A70000203306002019
:1015700004000020FC8B0008549800081C98000808
:10158000E89700085C9800089C980008C498000838
:10159000D0980008F8980008309900083899000899
:1015A000409900086499000888990008C0990008CB
:1015B000E09900080C9A000880980008149A000826
:1015C000DC8B000864980008DF00002016F8013F5B
:1015D000013507F8013F05F035F88542B348F5D3EA
:1015E00000231E46B24901220D44B24F85F8DC307B
:1015F00022704F200136B6B2FEF7BAFEB85D002861
:10160000F8D1FFF710BB2D2B3FF48CAEA0E6AA4912
:1016100001A804F0EFFF002800F09A81A74901A873
:1016200004F0E8FF002800F08781A54901A804F034
:10163000E1FF002800F07981A24901A804F0DAFF57
:10164000002800F06B81A04901A804F0D3FF002816
:1016500000F023819D4901A804F0CCFF002800F090
:1016600015819B4901A804F0C5FF002800F0058101
:10167000984901A804F0BEFF002800F0F5809649C3
:1016800001A804F0B7FF002800F0E780934901A803
:1016900004F0B0FF002800F0E080914901A804F0B8
:1016A000A9FF002800F0D2808E4901A804F0A2FF13
:1016B000002800F0C4808C4901A804F09BFF00289A
:1016C00000F0B680894901A804F094FF002800F0DA
:1016D000AF80874901A804F08DFF002800F0A180A9
:1016E000844901A804F086FF002800F09380824915
:1016F00001A804F07FFF002800F083807F4901A843
:1017000004F078FF002875D07D4901A804F072FF2D
:1017100000286FD07B4901A804F06CFF002862D03C
:10172000794901A804F066FF054600284BD07749A7
:1017300001A804F05FFF0546002834D0744901A8D1
:1017400004F058FF0546E8B1724901A804F052FFC1
:1017500030B1714901A804F04DFF002840F07581B7
:10176000524804F0DEFE524B524F83F887000025AA
:101770004F200135ADB2FEF7FBFD785D0028F8D1B2
:10178000FFF751BA494804F0CCFE494B494F83F862
:1017900086004F200135ADB2FEF7EAFD785D0028E6
:1017A000F8D1FFF740BA414804F0BBFE404B414F2F
:1017B00098774F200135ADB2FEF7DAFD785D00284D
:1017C000F8D1FFF730BA394804F0ABFE384B394F47
:1017D00058764F200135ADB2FEF7CAFD785D00287E
:1017E000F8D1FFF720BA324D287FFEF723FE287785
:1017F000FFF719BA2E4D687DFEF71CFE6875FFF7DE
:1018000012BA2B4D95F8FA00FEF714FE85F8FA008F
:10181000FFF709BA264D687FFEF70CFE6877FFF7E1
:1018200002BA234DE87CFEF705FEE874FFF7FBB92A
:101830001F4DA87CFEF7FEFDA874FFF7F4B91C4D00
:10184000687CFEF7F7FD6874FFF7EDB9184D287C4A
:10185000FEF7F0FD2874FFF7E6B9154DE87BFEF7BB
:10186000E9FDE873FFF7DFB9114D95F88900FEF740
:10187000E1FD85F88900FFF7D6B90D4D95F8880090
:10188000FEF7D8FD85F88800FFF7CDB9084DA87D93
:10189000FEF7D0FDA875FFF7C6B9054D95F8850090
:1018A000FEF7C8FD85F88500FFF7BDB934060020B6
:1018B00004000020FC8B0008349A00083C9A0008C1
:1018C000449A00084C9A0008549A00085C9A000850
:1018D000689A0008749A0008809A0008889A00089C
:1018E000949A00089C9A0008A49A0008A89A0008F4
:1018F000B49A0008BC9A0008C89A0008D49A000854
:10190000D89A0008E49A0008F09A0008FC9A0008A7
:10191000089B0008149B0008209B0008C34D287EEC
:10192000FEF788FD2876FFF77EB9C04DA878FEF750
:1019300081FDA870FFF777B9BC4D6878FEF77AFD96
:10194000BB49BC4B0122687008701A70FFF76BB975
:10195000B64D2878FEF76EFD2870FFF764B9B648DB
:1019600004F0DFFDC0B20F282DD8B04A0123B34FD9
:1019700082F8C700237000254F200135ADB2FEF775
:10198000F7FC785D0028F8D1FFF74DB9AA4804F0BC
:10199000C8FD642806DDAA4BC21783FB0013184458
:1019A000C2EB2020D8B1042819DCA04BA34F187338
:1019B00000254F200135ADB2FEF7DAFC785D002836
:1019C000F8D1FFF730B99F4E00256F200135ADB239
:1019D000FEF7CEFC705D0028F8D1FFF724B99A4ECF
:1019E00000253120FEF7C4FC681C85B2705D00281C
:1019F000F8D1FFF718B9904804F093FD934BA0F588
:101A000096729A42064639D8914AC31782FB001251
:101A10008649C3EB6213894FC1F8D43000254F21AA
:101A200001350846ADB2FEF7A3FC795D0029F7D178
:101A3000884802F0A5F83046012101F0EBF90121B8
:101A4000844802F09DF8FFF7EEB8834901A804F03E
:101A5000D1FD0646002835D001A8804904F0CAFD12
:101A60000546B8B17E4E00253F200135ADB2FEF7E8
:101A70007FFC705D0028F8D1FFF7D5B8794E0025BE
:101A800033200135ADB2FEF773FC705D0028F8D14C
:101A9000FFF7C9B8664A654B167818462A46FC21F6
:101AA0005E7000F033FA002840F0B5806E4E0546B7
:101AB00050200135ADB2FEF75BFC705D0028F8D117
:101AC000FFF7B1B843F6982E584D684FDFF8AC9148
:101AD0004FF0020AE8732874687428756877C5F8AF
:101AE00004E04FF0640B4FF0010E85F80CA085F870
:101AF0000EA085F81EA080460FCF4FF0070AC5F84C
:101B00001F000420C5F82310C5F82720C5F82B3086
:101B1000C5F808B0687685F800E00FCF85F801E0D9
:101B200085F802E085F812E085F813E085F815E005
:101B300085F816E085F818E085F80DA0DFF840B1CB
:101B4000C5F82F00D9F8000005F1A407C5F8331037
:101B5000C5F83720C5F83B30C5F88A0099E803007E
:101B60004FEA114CC5F89400A5F89810BBE80F0097
:101B70000FC7DBF800303E4999F80600B9F804B009
:101B800085F885E04FF03C0E3B803A4A0F8885F897
:101B900086E04FF0050E85F89AC085F887E005F1DC
:101BA000DC0385F8900085F8836085F8846085F80B
:101BB000886085F88960A5F88EB0DFF8C8C091F814
:101BC0000290DFF8C4E092E80300A5F8C27083E851
:101BD000030060220B211923184F85F8C49085F863
:101BE000D0A085F8FA602E7785F8C710C5F8C8C070
:101BF000C5F8CCE0C5F8D420C5F8D8304F2008F19E
:101C000001081FFA88F8FEF7B3FB17F80800002850
:101C1000F5D1FFF708B8184E43200135ADB2FEF7F5
:101C2000A7FB705D0028F8D1FEF7FDBF040000207F
:101C3000AC0600200801002034060020FC8B0008C0
:101C400049D6B9F2C899000890990008D4C001009B
:101C50001F85EB51004800402C9B0008789B000832
:101C6000BC9B0008E8990008809B0008309B000896
:101C70006C9B0008709B00089C9B0008509B000810
:101C8000589B00080040D8430040D943854804F0E1
:101C900048FCC0B2431E012B1CD9834E31200135B4
:101CA000ADB2FEF765FB705D0028F8D1FEF7BBBF53
:101CB0007C4804F036FCC0B2C31F012B17D97B4E01
:101CC00037200135ADB2FEF753FB705D0028F8D127
:101CD000FEF7A9BF764B774F98734F200135ADB211
:101CE000FEF746FB785D0028F8D1FEF79CBF704BED
:101CF000704F58734F200135ADB2FEF739FB785D58
:101D00000028F8D1FEF78FBF664804F00AFC4FF4B4
:101D10007A7303FB00F0664A664F50604F2001352E
:101D2000ADB2FEF725FB785D0028F8D1FEF77BBF4A
:101D30005C4804F0F3FB03F015F95F49064603F035
:101D400021FC20B15D49304603F008FC58B95C4ED7
:101D5000054646200135ADB2FEF70AFB705D00284E
:101D6000F8D1FEF760BF524B3046524FC3F8CC60FB
:101D700001F076FD4F200135ADB2FEF7F9FA785D3E
:101D80000028F8D1FEF74FBF464804F0C7FB03F028
:101D9000E9F84949064603F0F5FB38B347493046B0
:101DA00003F0DCFB10B3424B424FC3F8C8604F2036
:101DB0000135ADB2FEF7DCFA785D0028F8D1FEF708
:101DC00032BF384804F0ADFBA0F11903B3F58A7FA8
:101DD00018D2374B374F98604F200135ADB2FEF720
:101DE000C7FA785D0028F8D1FEF71DBF344E0546CE
:101DF00046200135ADB2FEF7BBFA705D0028F8D180
:101E0000FEF711BF2F4E32200135ADB2FEF7B0FA0A
:101E1000705D0028F8D1FEF706BF224804F081FB70
:101E200000EBD070C0F34703062B24D8204A214F83
:101E3000D3754F200135ADB2FEF79AFA785D0028D0
:101E4000F8D1FEF7F0BE174804F06BFB00EBD07042
:101E5000C0F34703062B19D8154A164F82F8833072
:101E600000254F200135ADB2FEF782FA785D0028DB
:101E7000F8D1FEF7D8BE144E30200135ADB2FEF7D2
:101E800077FA705D0028F8D1FEF7CDBE0E4E002522
:101E900030200135ADB2FEF76BFA705D0028F8D145
:101EA000FEF7C1BE340600206C990008489900086E
:101EB00004000020FC8B0008000070430080684490
:101EC00000990008D8980008A898000802F100635B
:101ED00003F57C431B68B3F1553F01D001207047E7
:101EE00010B4094C0023144459B1CA1A032A88BFFC
:101EF00054F8042B03F1040388BF40F8042B9942E3
:101F0000F3D8002010BC704704FC00082DE9F04114
:101F10000F461546064601F0F9FE342001F00AFF8F
:101F2000144801F07BFF80B2042802D00120BDE8F4
:101F3000F0814FF055310F4801F03CFF0E4C1FFA75
:101F400080F82C44354667B1204655F8041B01F053
:101F500031FF043401F0F4FE0428FBD1AB1B9F4297
:101F6000F2D801F0DFFEB8F1040018BF0120BDE88F
:101F7000F08100BF00FC000804FC00082DE9F041DE
:101F8000CC78E30648BF8B78098804F00F0748BF78
:101F90001F4311F0FF0F21D0066800234FF0010E00
:101FA0004FF00F0802E00133082B16D00EFA03F2AF
:101FB00032EA0105F7D19D0008FA05FC26EA0C0675
:101FC00007FA05F5282C46EA050631D0482C03F11E
:101FD000010308BF0261082BE8D10660FF2923D95D
:101FE000466800234FF0010E4FF00F0802E0013366
:101FF000082B18D003F108020EFA02F232EA0105AA
:10200000F5D19D0008FA05FC26EA0C0607FA05F54D
:10201000282C46EA050609D0482C03F1010308BF25
:102020000261082BE6D14660BDE8F0814261DEE73F
:102030004261B8E7016170474161704708B540F2FD
:1020400025510B4801F0D4FD48B94FF458710848A8
:1020500001F0CEFDBDE80840054801F0BFBD0448D1
:1020600001F0BCFDBDE80840C0B200F0F3BC00BF09
:102070000038014008B540F225510B4801F0B8FD89
:1020800048B94FF45871084801F0B2FDBDE8084066
:10209000054801F0A3BD044801F0A0FDBDE80840DB
:1020A000C0B2FEF789B900BF004800400000000040
:1020B000F8B501214FF08040FEF720F900B9F8BDD6
:1020C00001214FF08040FEF725F9694B1B78012B69
:1020D00079D0684C01F0DCF800285DD12379654E99
:1020E000002B3AD1644DEB78634E002B57D1EB783F
:1020F00061494BB9614A1368013B136023B901235D
:102100004B711368013B1360D4F80431013BC4F8F0
:1021100004313BB9A979584A01B901239371C82305
:10212000C4F804316379534A002BC8D192F80831BE
:10213000002BC4D052490B68013B0B60002BBED171
:102140004FF480714F4882F80831FFF773FFBDE804
:10215000F84080214B48FFF76DBF4B4F464D7B88C1
:10216000D6F800219BB2934239DCAB78002B54D1D6
:1021700000232B802B889BB2002BB4D1788880B2AF
:1021800002F050FC38A3D3E9002302F0B1FC02F0C6
:10219000C1FEC4F80001A6E701F074F8C2E73B4FA6
:1021A000386801F051FDB3783071002B9FD10228BF
:1021B00039D001284FD0002899D10146012273203F
:1021C00001F03EFB93E7FEF795F92A4C207018B911
:1021D0002F4B227F1A707DE701F03AF8F8E72B8841
:1021E000802101339BB227482B80FFF725FFF16840
:1021F000284B2A8883FB010392B2A3EBE1739A4236
:10220000B8DD01234FF480711E48AB70FFF712FF59
:1022100080211C48FFF70EFFACE74FF480511E48A9
:10222000FFF708FFA4E73B685A1C3A605B7803F0AD
:10223000FF02002B7FF45BAFE1684FF47A7393FBEE
:10224000F1F1A3680D48B3FBF1F3F2700360727112
:1022500001F05EFB4BE70246217C732001F0F0FAAF
:1022600045E700BFAFF300809A9999999999F13F9A
:102270009D07002000000020BE030020A0080020D1
:102280009C080020000C0140240600209808002033
:10229000B0070020565555550008014010B501F013
:1022A00063FB144B4FF416721B8813499BB202FB5D
:1022B00003F3124C124A1B1308702046138000F0DF
:1022C00039FB104A237D022BD3798CBF43F0800366
:1022D00003F07F03D3710C4B93F887200AB9DB7EA0
:1022E00033B121686068094ABDE8104002F0C4B902
:1022F00010BD00BF240600209C070020B40700206A
:10230000AE070020BE03002000000020A007002030
:102310002DE9F04F7E4BDFF850A287B028221A70CB
:10232000FFF7BCFFDAF800307A49DAF8042081FBC5
:10233000030781FB0201D817C0EBA75783EAE375B7
:10234000002FA5EBE375744BB8BF7F424FEAE278EC
:1023500003FB0755C8EBA151002A81EAE178B8BF19
:102360005242A8EBE17803FB0823002D6B4CB8BF69
:102370006D42A4FB0525002B694EDFF8F0B1DFF8B4
:10238000F091B8BF5B42A4FB0334AD09DBF8003029
:1023900006F1980248466349059504F007F9B37EB3
:1023A000A4090546002B62D15F48DAF804305F4A81
:1023B000039412EA230138BF0146DAF80040059B76
:1023C0000191009312EA240238BF02463B4609EB12
:1023D0000500CDF80880564904F0E8F8B37D0544BF
:1023E000002B40F08680337D002B79D1F37E002BCB
:1023F0006ED1F37C002B61D1F37D002B4DD1737E28
:10240000002B41D14B494FF6FF7311F8012FB2B1A8
:1024100083EA0223082213F4004F4FEA430318BF54
:1024200083F4815302F1FF3218BF83F0010312F0ED
:10243000FF029BB2EFD111F8012F002AE8D11A4612
:102440003D4909EB0500A6F80A3104F0AFF83B4B13
:10245000C3F8009001F074FADBF80030384A013319
:102460000121CBF80030D17007B0BDE8F08F9AF8A9
:1024700011109AF8123000919AF81320314948440B
:1024800004F094F805448FE709EB05009AF8102052
:102490002D4904F08BF80544B4E72C4B2C4A1B88DB
:1024A0006FF06301A2FB0302520901FB023309EB47
:1024B0000500284904F07AF80544A0E7264B09EB0B
:1024C0000500214993F9002004F070F8054493E7D2
:1024D00009EB0500214A224904F068F8054488E721
:1024E00009EB0500DAF80C201E4904F05FF80544FA
:1024F0007CE7DAF808300949DA1781FB031309EBA6
:1025000005001849C2EBA31204F050F805446AE72D
:10251000280900206BCA5F6B806967FFD34D62108A
:1025200000000020EC9B0008F0940008E89B0008E5
:10253000089C0008D30700203C9C00089808002055
:10254000BE030020F89B00082C9C0008AE0700206A
:102550001F85EB51309C00089C070020A00700203D
:10256000289C0008209C0008B40700209807002041
:10257000D0070020F0B5164C164D87B0204600213C
:1025800001F0FEFA2846002101F0FAFA01F0D8F92C
:10259000FFF784FE104A114B114992F9006003F1D4
:1025A00010020F8807CA8DE8070004970FCB039627
:1025B00000F074FE01F0ACF92846012101F0E0FAC8
:1025C0002046012107B0BDE8F04001F0D9BA00BFB4
:1025D00000380140004800409C070020B40700205C
:1025E000AE070020F8B5284D284F294E00237B71F7
:1025F000FFF754FE05F1A8023046264903F0D6FF46
:1026000095F887300446002B37D195F88C3033BBD2
:1026100095F88D3073B1204B204A1B886FF0630111
:10262000A2FB0302520901FB023330191C4903F0DB
:10263000BDFF04441B4B012218889D7833191146B5
:1026400030539D70732001F0FBF8114801F012FD2A
:102650004FF4FA60FDF7C2FD01237B71F8BD124B08
:10266000124A9B68124982FB0302DB173019C3EB45
:10267000A21203F09BFF0444CAE70E4A0E49301829
:1026800003F094FF0444C0E700000020BE030020D4
:10269000D0070020489C0008AE0700201F85EB51A2
:1026A000589C0008689C0008B4070020D34D6210B5
:1026B0004C9C0008A0070020449C00082DE9F0472E
:1026C000584F00F001FC00F0F9FB00F065FC4FF4FE
:1026D00080715548FFF7AEFC0022FC21381DFFF742
:1026E000F5FBF86800F072FDFDF71CFD00F000FA44
:1026F000D7F8D830642000FB03F0012100F08AFBFA
:10270000FA684FF4167303FB02F3DFF83081474A8F
:1027100001214748136001F033FAC646454C04F1E5
:10272000300625460FCDB542CEF80000CEF8041095
:10273000CEF80820CEF80C3004F110040EF1100E83
:10274000EFD103CC3C4D23782E46CEF800008EF816
:102750000830CEF804103948FDF720FE01F0ECF8FF
:10276000D7F8D00001F07CF897F8D410012201F0DE
:1027700007016D2001F064F801220021712001F0B1
:102780005FF80122F021132001F05AF80122002104
:10279000122001F055F8012280210F2001F050F89D
:1027A000DFF8A090264A3B7F0021E9700121C2F8A2
:1027B0000080697189F80030DFF868A000F048FDFA
:1027C0007C7F97F88B80EB789BB973798BB1B4B130
:1027D00097F8893023B108F1FF3818F0FF081BD0B3
:1027E000BB79A3B1FFF794FDEB78013CE4B2002B79
:1027F000EBD00021102001F031FC30BFE3E799F865
:1028000000307C7F002BDED0FFF7B4FEDBE7DAF888
:102810000800FDF7E3FCE7E7FFF7E4FE9AF88B809A
:10282000DEE700BF00000020000C01409C080020F3
:10283000004800406C9C0008BE030020D007002028
:1028400098080020B007002010B504464021084831
:1028500001F0C8F90028F9D02146054801F0BAF97D
:102860004021034801F0BEF90028F9D010BD00BF97
:10287000003801402DE9F04F98468B464118C9B207
:10288000DBB2CD18EDB24FEA182A05EB0A07014476
:102890000D44FFB23D4483B08146EDB2B8F1000F64
:1028A00033D016460024325D01341744FFB2E4B23F
:1028B0003D44A045EDB2F6D8B5200193FFF7C4FF23
:1028C0006220FFF7C1FF4846FFF7BEFF5846FFF7FB
:1028D000BBFF019B08F1FF381846FFF7B5FF5046D4
:1028E000FFF7B2FF1FFA88F8B044741E14F8010F06
:1028F000FFF7AAFFA045F9D13846FFF7A5FF284604
:1029000003B0BDE8F04FFFF79FBFB5200193FFF77D
:102910009BFF6220FFF798FF4846FFF795FF584658
:10292000FFF792FF019B1846FFF78EFF5046FFF717
:102930008BFFE1E730B4054672B6064C0FCC286039
:102940006960AA60EB6007CC28616961AA6162B620
:1029500030BC7047A4080020F0B58578C67884881C
:10296000AB19DBB21A19D2B202EB14212B441A4470
:10297000C9B20A44D2B200F1060E54B100231EF8C7
:10298000037001333944C9B2DBB20A449C42D2B26B
:10299000F5D81EF8043074448B4204D02B4A138BB4
:1029A00001331383F0BD63789342F7D1012D02D038
:1029B000052D10D0F0BD072E23D0022E13D0062EE9
:1029C0003AD0212EF6D1214B847DC17D027EDC746C
:1029D00099745A74F0BD012E35D0002EEAD11C4BEB
:1029E00001225A70E6E7194BDA8A0132DA82D0F80E
:1029F0000E201A60D0F80A205A60D0F816209A608B
:102A0000F0BD124B817EDA8A19750132DA82D0F874
:102A10002210827B1960D0F81E40417F5C60D0F8A4
:102A20002A40DA74C27B9C609A74027C19745A74CE
:102A3000D0F84220DA60F0BD044B017C90F83520DC
:102A400019751A74F0BD024B1E70F0BDA408002069
:102A5000C803002010B5184CA37833B9E378BBB98C
:102A6000B52825D00023E37010BDE378E218042BCD
:102A7000107104D92289591E0832914211D00133B4
:102A8000DBB2632B89BF0023E370E370A37010BD3A
:102A9000012BE7D16228E5D10222A3706071E270B8
:102AA00010BD201DFFF758FF0023E370A37010BD79
:102AB00001232071E37010BDC803002070B50B4DD9
:102AC00000232B702E466B70C92407E073784BB936
:102AD000FDF784FB631E13F0FF0403D02B78012065
:102AE000002BF3D02878C0B270BD00BFC80300200F
:102AF0002DE9F0476225FEB02A46002101A803F027
:102B00004CFD4FF6FF73012406262146B5274FF0F2
:102B100004084FF41640ADF80A308DF80C408DF8DB
:102B200005508DF804708DF806608DF80780ADF8BB
:102B3000088000F01BF90A20FDF750FBBDF80830B3
:102B40000DF10A029DF807109DF80600FFF792FEAE
:102B50004FF44870FDF742FB21464FF4165000F049
:102B600005F90A20FDF73AFBBDF808300DF10A021D
:102B70009DF807109DF80600FFF77CFE4FF44870A3
:102B8000FDF72CFB2A4600211AA803F006FD4FF0A2
:102B9000000914224FF40C61134630464FF4164AD4
:102BA000ADF87210ADF86C2049460DF16E028DF84B
:102BB0006E40ADF87A40ADF87C408DF868708DF8C5
:102BC00069508DF86A60ADF87490ADF87890ADF802
:102BD00076A0FFF74FFE2146504600F0C7F80A20C6
:102BE000FDF7FCFA49462A4633A803F0D6FC112427
:102BF00002224FF0080E3046214613468DF8D3804E
:102C00008DF8CC708DF8CD508DF8CE608DF8D2E077
:102C10008DF8CF40ADF8D02005E09DF8CE009DF8AE
:102C2000CF10BDF8D0300DF1D202FFF723FEFFF731
:102C300045FF0028F1D06226324600214CA803F05F
:102C4000ACFC062501220324B5278DF8316102264C
:102C50002846114623468DF832518DF833218DF8E0
:102C600036218DF83821ADF834418DF830718DF86A
:102C7000376105E09DF832019DF83311BDF834311C
:102C80000DF59B72FFF7F6FDFFF718FF0028F1D056
:102C900006238DF83731BDF834310DF59B729DF860
:102CA00033119DF83201FFF7E5FDFFF707FF00281C
:102CB000F1D021238DF83731BDF834310DF59B72F9
:102CC0009DF833119DF83201FFF7D4FDFFF7F6FEB2
:102CD0000028F1D040F2FF3742F2107662252A46F2
:102CE0000624002165A803F058FC242220468DF814
:102CF00095518DF8964107250224134611464FF051
:102D0000B50E8DF89721ADF89821ADF89A7119227A
:102D10000027ADF8A2618DF89C51052664258DF839
:102D20009D418DF8B1414FF496748DF894E1ADF862
:102D3000A4718DF8A661ADF8A821ADF8AA21ADF86F
:102D4000AC51ADF8AE4105E09DF896019DF89711A4
:102D5000BDF898310DF5CD72FFF78CFDFFF7AEFE93
:102D60000028F1D07EB0BDE8F08700BF2DE9F0412A
:102D700080460F46244D202682B0002240F2255185
:102D80002248C5F8846000F009FF40F225511F4831
:102D900000F052FF4FF458711C4800F04DFF002125
:102DA0001A4800F0EDFE01214FF4804000F0EAFCEB
:102DB000174B002219460C2414485C819A80DA8053
:102DC0001A819A81C3F80080012400F07BFE25213E
:102DD0000F22022301A88DF804108DF805208DF82C
:102DE00006308DF8074001F0F9F82146074800F059
:102DF000C7FE37B1224640F22551044800F0CEFE0E
:102E00006E6002B0BDE8F08100E100E000380140F2
:102E1000EC0800202DE9F04180460F46244D802625
:102E200082B0002240F225512248C5F8846000F0AB
:102E3000B5FE40F225511F4800F0FEFE4FF45871D8
:102E40001C4800F0F9FE00211A4800F099FE01210B
:102E50004FF4802000F0A4FC174B002219460C24EC
:102E600014485C819A80DA801A819A81C3F80080C4
:102E7000012400F027FE27210E22022301A88DF84D
:102E800004108DF805208DF806308DF8074001F00C
:102E9000A5F82146074800F073FE37B1224640F2FC
:102EA0002551044800F07AFE6E6002B0BDE8F08162
:102EB00000E100E000480040EC08002000214FF055
:102EC000006001F0C1B800BF10B500F065FB4FF421
:102ED000803000F085FB00F09FFB012800D010BD82
:102EE0000446102000F006FF022000F0F9FE9020BA
:102EF00000F0BEFB4FF4A06000F0CEFB4FF480600A
:102F000000F0C0FB204600F0A1FB00F0A9FB042864
:102F1000FBD110BD1C4B2DE9F0414FF400420126BE
:102F200019464FF018081948194C1A4D1A8083F8A1
:102F300003809E70FFF722F831464FF4804000F086
:102F40002FFC4FF40060002307224FF482772146C4
:102F5000A080284622822380E3802381E381A4F895
:102F60000C80678001F014F93146284601F044F9DD
:102F70003146284601F02CF9284621466780BDE8F5
:102F8000F04101F005B900BFD4080020000C014059
:102F9000D8080020003800402DE9F84F754C012179
:102FA0000420012500F0EEFB10264FF4805321464B
:102FB00071482380E670A570FEF7E0FF29460820DF
:102FC00000F0E0FB4FF4C07321466C484FF0180846
:102FD000E6702380A570FEF7D1FF4FF42043214611
:102FE00066480427238084F80380A570FEF7C6FF97
:102FF0004FF48043214661482380E770FEF7BEFF0F
:103000003046294600F0BEFB4FF4005B21465C4889
:10301000E6704FF4007AA570A4F800B0FEF7AEFF9A
:10302000FFF778FF214654484FF4806984F8038005
:10303000A570A4F800A0FEF7A1FF21464E48E77056
:10304000A4F80090FEF79AFF00214FF41650FFF706
:103050008DFE2146494884F80380A4F80090A570AD
:10306000FEF78CFF4FF40063214644482380E7704D
:10307000FEF784FF00214FF49640FFF7CBFE294670
:10308000284600F071FB3F483F4E00F0E7FE3F4B03
:1030900000274FF0020829463D487360C6F80C80AF
:1030A000B760B76200F09CFC3A4A80204FF480730E
:1030B000C6F81C9031464FF02009706131483260EB
:1030C000B3613761C6F824B0C6F8209000F05AFF0B
:1030D00029462C4800F076FF4023214626482380CD
:1030E000E770FEF74BFF21462348A4F80090E770F5
:1030F000FEF744FF384600F0D9FA2946504600F062
:1031000041FB254B4FF46022194621489A601F600D
:103110001D715D71DF6083F8108000F033FC2A467A
:10312000032305211A4800F083FC424603230621AD
:10313000174800F07DFC2946154800F051FC144862
:10314000294600F043FC124800F054FC104800F0FF
:1031500057FC0028FAD10E4800F056FC0C4800F04D
:1031600059FC0028FAD101210948BDE8F84F00F0C8
:1031700055BC00BFD408002000080140000C0140ED
:103180000010014008000240FC0800202406002036
:10319000002401404C240140C008002038B50848F4
:1031A00000F0C0FF074B4FF40045102401221946E0
:1031B0001D80DC709A700448BDE83840FEF7DEBE22
:1031C00000380040D4080020000C014030B504460F
:1031D000012185B0084600F0E3FA0021012000F04B
:1031E000FBFA1A4B052293FBF4F301A90024013BDF
:1031F0004FF08040ADF80830ADF80420ADF806403F
:10320000ADF80A408DF80C40FDF706F801214FF0AB
:103210008040FDF77FF8012211464FF08040FDF716
:1032200067F801251C2368468DF800308DF80140B1
:103230008DF802508DF8035000F0D0FE29464FF073
:103240008040FDF73DF805B030BD00BF40420F00A3
:1032500030B5094B094893F83D5085B003F152044D
:1032600000223021019002910095039411460448F8
:1032700001F0E6F805B030BD8E000020A89C0008E3
:1032800034040020014801F033B900BF34040020A9
:10329000014B93F86C0170473404002084B02DE991
:1032A000F04FAE4DB5B03EAE86E80F0085FB002373
:1032B0009DF91421C117C1EBA3031092BDF8182189
:1032C000002BDDF800A1119240F3FD800446A44DCF
:1032D000A44A85FB0404C1EBA45465B202FB053388
:1032E000A14F03EB43035B0087FB03279F49DA17DA
:1032F00081FB0313C2EB673707EB8701C2EBA31314
:10330000C7EBC10203EB8203DBB212933F99934BED
:10331000C81783FB0123C0EBA303002B40F3AE804F
:103320008F4C904A84FB0141C0EBA1514CB202FB8F
:1033300004338D4E03EB43035B0086FB03268B496E
:10334000DA1781FB0313C2EB663606EB8601C2EB8C
:10335000A313C6EBC10203EB8203DBB21393DFF8C6
:1033600030B2DFF814929BF80020DFF82882B9F819
:103370007431013298F81E10D2B201339BB28A42E6
:10338000A9F874318BF8002024D319B309F5BC7364
:10339000184608F11F010F9303F04CF998F81C3000
:1033A000002B40F0B580714B4FEAEA7283FB0A3A7A
:1033B000C2EBAA1A98F81D30002B40F0BE8098F896
:1033C000FA30002B40F0B2800022B9F874318BF84B
:1033D00000200BE0654A4FEAEA7182FB0A2A0022CC
:1033E00089F87821624AC1EBAA1A0F92002D84EA6B
:1033F000E471D4BF53204E20A1EBE471002C4FF4B4
:103400004D6404FB0AFA594C099384FB0A24119A6F
:10341000139BF6B203960C920F9E109A98F8C2E096
:1034200098F8C3C004934FEAEA7A129BD4BF4FF0D6
:1034300057094FF045090D960B929DF80861CAEBAC
:10344000A41485EAE57200930190FBB20291A2EB0D
:10345000E572CDF81CE0CDF818C00894CDF81490B2
:1034600014A844490A9603F0A1F814A9424801F0AF
:10347000E9F835B0BDE8F04F04B070473F4C5A4210
:1034800084FB0214D217C2EBA444364A61B202FB99
:1034900001F2D31A03EB4303334E5B0086FB032692
:1034A0003249DA1781FB0313C2EB663606EB86015D
:1034B000C2EBA313C6EBC10203EB82036442DBB28F
:1034C00064B213934BE72D4D5A4285FB0215D21778
:1034D000C2EBA545234A69B202FB01F2D31A03EB02
:1034E0004303214F5B0087FB03272049DA1781FB49
:1034F0000313C2EB673707EB8701C2EBA313C7EBDC
:10350000C10203EB82036D42DBB26DB21293FDE6A2
:10351000164B4FEAEA7283FB0A3A0F98C2EBAA1ADB
:1035200053460246164903F041F843E7104A109B00
:103530001046144903F03AF846E71198124B024638
:10354000A3FB022364215B0901FB1301084A89B232
:10355000009110460D4903F029F830E7676666666A
:103560006BCA5F6BC0BDF0FF89B5F814D34D621014
:10357000AC050020EC9C00083404002083DE1B43D3
:10358000C09C0008E09C00081F85EB51CC9C000803
:103590000E010020040000200F4B10B419680F4AE0
:1035A00041F0010119605C684FF41F0022405A602D
:1035B0001A68002122F0847222F480321A601A689C
:1035C00010BC22F480221A605A6822F4FE025A606B
:1035D0009860D962704700BF001002400000FFF8F9
:1035E0000C4BB0F5803F1A6822F480321A601A68DA
:1035F00022F480221A6008D0B0F5802F04D11A6816
:1036000042F4A0221A60704770471A6842F4803270
:103610001A6070470010024082B000230A4A0193EA
:1036200002E0B3F5A06F08D0136813F4003F019BCC
:1036300003F101030193019BF3D0034B1868C0F31E
:10364000404002B0704700BF00100240034A536878
:1036500023F0030318435060704700BF001002407E
:10366000024B586800F00C00704700BF0010024089
:10367000034A536823F0F00318435060704700BFBB
:1036800000100240034A536823F4E063184350607B
:10369000704700BF00100240034A536823F4605390
:1036A00043EAC0005060704700100240034A53686C
:1036B00023F4404318435060704700BF001002409D
:1036C000244910B44B6803F00C03042B33D0082BAF
:1036D00025D00BB3204A134602601E4A1F49546886
:1036E000C4F303140C5DE34043605468C4F3022444
:1036F0000C5D23FA04F484605468C4F3C2240C5DA6
:10370000E340C360526810BCC2F381320A44127CA9
:10371000B3FBF2F3036170470F4B0360DDE74B68C7
:103720004C68C3F383439A1CE30307D40C4B03FB9D
:1037300002F30360D1E70B4B0360CEE7CB6A094984
:1037400003F00F030133B1FBF3F302FB03F3036058
:10375000C3E700BF0010024000127A0010010020F1
:1037600000093D0000366E0129B9054A536923EA74
:10377000000050617047024B5A691043586170470E
:103780000010024029B9054A936923EA00009061BC
:103790007047024B9A6910439861704700100240CD
:1037A00029B9054AD36923EA0000D0617047024B6A
:1037B000DA691043D86170470010024029B9054A00
:1037C000D36823EA0000D0607047024BDA681043E8
:1037D000D86070470010024029B9054A136923EAEE
:1037E000000010617047024B1A691043186170475E
:1037F0000010024010B54FF4005104460E48FEF789
:103800001BFC02210D4800F005FD0028F9D02146DF
:103810000A4800F0EBFC0121084800F0FBFC0028FE
:10382000F9D04FF400510448FEF704FC034800F0BF
:10383000DFFCC0B210BD00BF0010014000380040E6
:103840002AB9000200B2084380B2FFF7D3BF40F0AC
:103850008000000200B2084380B2FFF7CBBF00BF78
:1038600070B52549064601F0DBFC2449044601F009
:1038700089FE2349051C204618BF012501F084FD5F
:1038800001F0BAFEAC00C0B22C1B183800EBC40328
:10389000681C93FBF0F401F06FFC1A4901F0C0FCC6
:1038A0000146304601F070FD0646E0B201F064FCCE
:1038B0000146304601F0AAFB134901F0A7FB13496A
:1038C00001F0AEFC01F098FE04F01F0444EA451438
:1038D00085B244F4754040F04000FFF78BFF280AA2
:1038E00040F47640FFF786FFE8B240F47740BDE849
:1038F0007040FFF77FBF00BF3BB1933F0000F04334
:1039000000002041ABAA0A410000C04100007A47F4
:1039100008B548F24070FFF76DFF054B1B7803B9FF
:1039200008BD4FF480710348BDE80840FEF782BB34
:1039300008010020000C014048F28070FFF75ABFD8
:1039400008B548F24B70FFF755FF054B1B7803B9DC
:1039500008BD4FF480710348BDE80840FEF76CBB1A
:1039600008010020000C014010B541F2FF10FFF7E4
:1039700041FF044648F68070FFF73CFF6010503866
:1039800040B210BD42680B6822F4702230B422F4B9
:1039900080720C79134343EA042343608568CC6842
:1039A0008A68094B22432B404C79134343EA440372
:1039B00083600A7CC36A013AD2B223F4700343EAFB
:1039C0000253C36230BC7047FDF7F1FF836819B939
:1039D00023F001038360704743F001038360704765
:1039E000836819B923F480738360704743F480734C
:1039F00083607047836843F008038360704700BFAB
:103A00008068C0F3C0007047836843F0040383609C
:103A1000704700BF8068C0F380007047836819B9A1
:103A200023F4A0038360704743F4A00383607047CE
:103A3000092970B41DD9A1F10A0606EB4606C5682E
:103A40000724B440B34025EA04042343062AC36094
:103A50001BD90C2A27D90D3A02EB8202C36A1F2414
:103A6000944001FA02F223EA04010A43C26270BCE4
:103A7000704701EB410605690724B440B34025EACD
:103A800004042343062A0361E3D8013A02EB8202CD
:103A9000436B1F24944001FA02F223EA04010A4313
:103AA000426370BC7047073A02EB8202036B1F242B
:103AB000944001FA02F223EA04010A43026370BC53
:103AC000704700BF30B504460D46038ACA889BB2D2
:103AD00023F440531343038282890B89888892B26E
:103AE0004989034322F4B0520B4322F00C021343E2
:103AF0009BB2A381A38AAA899BB223F4407387B0A7
:103B00001343A38201A8FFF7DBFD04991A48039B26
:103B1000A289844208BF0B4612F4004F2A6803EBC7
:103B2000830314BF5200920003EB8303B3FBF2F351
:103B3000124DA189A5FB03206422400900FB12332A
:103B40000A044FEA00100AD41A013232A5FB0223FC
:103B5000C3F3431303439BB2238107B030BDD900A5
:103B60003231A5FB0131C1F3421242EA00039BB29C
:103B7000238107B030BD00BF003801401F85EB51E5
:103B8000838929B923F400531B041B0C83817047DC
:103B90009BB243F400538381704700BF10B401F01F
:103BA0001F04C1F342110123012903FA04F30FD0CA
:103BB00002290CBF103014302AB9026810BC22EA66
:103BC000030303607047026810BC1343036070472F
:103BD0000C30F1E7C1F30801818070478088C0F3A1
:103BE000080070470388194214BF01200020704765
:103BF000C1F3421210B4012301F01F04012A03FA99
:103C000004F315D0022A0CBF028A828A92B21340B2
:103C1000028892B24BB10123090A03FA01F10A4268
:103C200014BF1846002010BC7047184610BC7047DF
:103C3000828992B21340EBE7090A012303FA01F1EA
:103C4000C94389B20180704730B41A491A4D0C78C3
:103C50002A78631CDBB20B70D2B9012B1DD0174A36
:103C6000557B0BD9072D1BD0092B07D830BC00780A
:103C7000023B40FA03F303F00100704795B90A2BA9
:103C800016D0927B92B900230B70022030BC704793
:103C9000013A2A70012030BC7047104630BC704792
:103CA000082BE3D9A31CDBB20B70E8E70B2BEAD19E
:103CB0000120EBE710060020280900200400002066
:103CC000044A05491368002B08BF0B4618441060CE
:103CD000184670471406002030090020FEE700BF98
:103CE000034A136803F0380318431060704700BF9D
:103CF00000200240044B1A6822F010021A601A6871
:103D000010431860704700BF00200240024B034977
:103D1000034A59605A6070470020024023016745FA
:103D2000AB89EFCD024A136943F0800313617047FA
:103D300000200240014BD860704700BF00200240C5
:103D4000084BDA68D1070BD4DA68520701D5022094
:103D50007047DB6813F0100F14BF03200420704776
:103D60000120704700200240084BDA68D1070BD4CD
:103D7000DA68520701D502207047DB6813F0100F94
:103D800014BF032004207047012070470020024028
:103D900010B50446FFF7E8FF012806D13CB1FFF754
:103DA000E3FF012804F1FF34F8D004B110BD052071
:103DB00010BD00BF70B5002382B005464FF400501F
:103DC0000C460193FFF7E4FF042801D002B070BD58
:103DD000114EA3B232694FF4005042F00102326139
:103DE0002B80FFF7D5FF042806D041F6FE73326919
:103DF0001340336102B070BD02350195019B240C64
:103E00001C804FF40050FFF7C3FF41F6FE73326988
:103E100013403361DAE700BF0020024038B50546A1
:103E20004FF43020FFF7B4FF042800D038BD0A4C0F
:103E30004FF43020236943F0020323616561236955
:103E400043F040032361FFF7A3FF41F6FD732269AE
:103E50001340236138BD00BF002002404FF6FE72C0
:103E600003683A491A4088424FF000030260036039
:103E700043608360C36027D0354B98422AD0354BCE
:103E800098422DD0344B984230D0344B984239D0A0
:103E9000334B98423CD0334B98420FD0324B984230
:103EA0003CD0324B98423FD0314B984242D0314BBC
:103EB000984245D0304B98421ED070472F4A5368E5
:103EC00043F07063536070472C4A536843F00F030C
:103ED00053607047294A536843F0F00353607047BA
:103EE000264A536843F4706353607047234A53680B
:103EF00043F4704353607047214A536843F470237E
:103F00005360DAE71D4A536843F4702353607047E7
:103F10001A4A536843F4700353607047184A536851
:103F200043F00F0353607047154A536843F0F003A2
:103F300053607047124A536843F47063536070478C
:103F40000F4A536843F470435360704708000240BF
:103F50001C00024030000240440002405800024071
:103F60006C00024080000240080402401C04024031
:103F70003004024044040240580402400000024061
:103F8000000402400A6A70B48D680B692A434D69C7
:103F900013438A691D43CB6945EA020402684D6AEE
:103FA00023438C6A1D4322F4FF43CE684A682C43A6
:103FB00023F070030D682343036046608560C26090
:103FC00070BC704729B94FF6FE7302681340036056
:103FD0007047036843F0010303607047C3785BB91F
:103FE000037801215A09164803F01F03203201FA11
:103FF00003F340F822307047124B30B4D96882780E
:10400000C9434478C1F302210F23C1F10405CB4019
:10401000AC401340027823431B0102F16042DBB243
:1040200002F5614282F800330378012203F01F0099
:1040300003495B09824041F8232030BC704700BF30
:1040400000E100E000ED00E021F0604121F07F019F
:10405000014B08439860704700ED00E0044A136983
:1040600019B923EA000010617047184310617047C6
:1040700000ED00E02DE9F84340F6B835274B047811
:1040800093F8863095FBF3F5002C44D06E0007467C
:10409000DFF88C8005EB06090CE0A4F12B032F2B35
:1040A0002BD94846FCF79AF83046FCF797F817F8F2
:1040B000014F74B302F04AFA2044437803F003033B
:1040C000022B08BF203CE4B2212CE6D1732409E086
:1040D0002846FCF783F8FFF71BFC2846FCF77EF820
:1040E000012CE1D0FFF72CFC14F0010F4FEA54042F
:1040F000EED03046FCF772F8EAE7444414F82B4C53
:10410000012CEFD83046FCF769F817F8014F002C66
:10411000D0D1BDE8F883BDE8F88300BF04000020DB
:10412000289D000808B5174B984212D0164B9842AC
:104130001BD0164B984200D008BD01214FF400401F
:10414000FFF74AFBBDE8084000214FF40040FFF7AD
:1041500043BB01214FF48050FFF730FBBDE808401E
:1041600000214FF48050FFF729BB01214FF480401C
:10417000FFF732FBBDE8084000214FF48040FFF715
:104180002BBB00BF0030014000380040003C004025
:104190004A8830B40C888B882243CC881A430B8918
:1041A00022434C898D891A4322430388CC892A43B0
:1041B000224303F4415313439BB20380838B0A8A47
:1041C00023F400631B041B0C838330BC0282704702
:1041D000038829B923F040031B041B0C038070479C
:1041E0009BB243F040030380704700BF818170475A
:1041F000808980B2704700BF838829B923F0040307
:104200001B041B0C838070479BB243F00403838024
:10421000704700BF0389194214BF01200020704776
:10422000A1F17E02B2FA82F22DE9F8432F4C00236D
:1042300052098946054626461F46227063704FF094
:10424000010811E0002B38D086F803800121B5F871
:104250007001FBF7A1FF63784FEA59090133DBB224
:10426000072B63703AD8327809F00103A370002A53
:10427000E8D12A8882EA0301C9074FEA520244BF03
:1042800082F4044282F008022A80B3B1E378013359
:10429000DBB2052BE370D9D10121B5F87001FBF732
:1042A0007BFF95F86931022B1AD0022385F869311A
:1042B000CA23A5F86E31E770C8E795F86931E77051
:1042C000022B06D0022385F86931CA23A5F86E3186
:1042D000BCE785F8698140F28913F7E7BDE8F88308
:1042E00085F8698140F28913E3E700BF18060020D2
:1042F00010B50446104BD3F8C800FFF7B1FA0122FD
:1043000005217220FFF79CFA4FF400510B48FDF78E
:1043100091FE012212217120FFF792FAFEF73EFF73
:10432000B4F80401012384F86C3100B910BDBDE874
:104330001040FBF753BF00BF0400002000100140F5
:1043400070B50646094C0025FEF7E4FDD4F8CC0014
:1043500086F86C51FFF784FA294601227120FFF795
:104360006FFAA068BDE87040FEF730BF040000207F
:1043700038B503880446D9436FEA1323084DC9B200
:104380002B71FFF74DFF29792046FFF749FF2046A3
:104390007E21FFF745FF2046BDE83840FFF7D0BF3C
:1043A00018060020F8B508460D46164602F04AF9F0
:1043B000C0B2002842D000273C46691E202200F1EE
:1043C000FF3E0CE02D2D08BF2025774504F10103A9
:1043D00035551CD0DCB20137FBB2984214D911F824
:1043E000015F2C2DEED12346062B13D8C3F1070411
:1043F000E4B21C44E4B25D1CF254EBB29C42FAD12C
:104400000137FBB29842EAD800233355F8BDDBB23E
:10441000062BEBD9A3F10804E4B2052C03D8C3F1B1
:104420000E04E4B2E5E7A3F10F04E4B2052C03D8CF
:10443000C3F11504E4B2DCE71C46CCE70446E3E72D
:104440002DE9F04740F21B3640F2891504469A46A2
:104450001B4F192380F868110121B860A0F8706122
:10446000C2708370A0F86E51A0F8041180F86A1130
:104470004FF020359DF82090DDF824809DF82870BD
:104480000B9EFFF75DFF04F583705146C4F806519B
:10449000858002F0CFF804F20D1084F80C91C4F876
:1044A0000D514146858002F0C5F884F813713146FC
:1044B00004F58A722046BDE8F047FFF773BF00BFDE
:1044C0001806002090F86B313BB9012380F86B315E
:1044D0004FF400410548FDF7ADBD002380F86B3176
:1044E0004FF400410148FDF7A7BD00BF000C01409B
:1044F00010B50446FFF7E6FF4FF080421388002115
:1045000023F001031B041B0C1380B4F86E31938558
:10451000918413889BB243F00103138010BD00BF48
:1045200038B50546FFF7E4FE2846FFF7E1FF4FF6F2
:10453000FF71AB780122298085F869214BB10024F5
:104540007E212846FFF76CFE0134AB78E4B2A3422B
:10455000F6D838BD70B514460D460646FFF7E0FFA5
:1045600034B115F8011B3046FFF75AFE013CF8D173
:104570003046FFF7FDFE002070BD00BF2DE9F04F73
:1045800004469B46904683B04FF0203A9DF8303069
:1045900000F10B02C0F80BA0251D1046A4F80FA0D7
:1045A00006220193DDF834900E9F0F9E02F052F820
:1045B00059460622C4F804A02846A5F804A002F033
:1045C00049F8B8F1400F88BFA8F10608019B88BFE1
:1045D0005FFA88F8A37284F81180484602F032F836
:1045E0008046421C494604F1120001F0CBFF5FFAFD
:1045F00088F000F10E080023E1180A790133DBB2DC
:10460000520043450A71F7D300F10D0323441A7990
:1046100004EB080E42F001021A71032223188EF8EF
:1046200004201030F0223946DA742844324602F071
:1046300011F829462046B21C424403B0BDE8F04FB1
:10464000FFF788BF30B5044685B008460D4601F037
:10465000F9FF94F8131104F58A7394F80C218DE88E
:104660002A00039004F20D1304F583712046FFF72E
:1046700085FF05B030BD00BF002A74D02DE9F04F92
:10468000904600EBD07085B043100393374B0291F6
:1046900093F88370012301934FF00009B9F1000FE3
:1046A0004CD0029800F068FD314900F06DFE3149B0
:1046B00000F0AEFC0546002F36D01227002401265C
:1046C00001E02D4B1F5D07FB06F6304600F09AF91E
:1046D00002460B460020294900F034FB00F042FC62
:1046E00001468346284600F04FFE00F085FF5FFA42
:1046F00080FA504600F040FD594600F091FD014619
:10470000284600F083FC0A2F14BF4122302208EB18
:104710004403924403F809A0144B013493F88370C6
:10472000E4B2A7420546CCD8019B022B12D100234C
:10473000012008F8173005B0BDE8F08F039800F0AD
:104740001BFD0B4900F020FE0A4900F061FC054604
:10475000002FB2D1019B09F1010903F1010A5FFAAF
:104760008AF301939AE71046704700BF04000020C7
:104770008096184B0000B442589D000800806640A7
:1047800081F0004102E000BF83F0004330B54FEA02
:1047900041044FEA430594EA050F08BF90EA020F6F
:1047A0001FBF54EA000C55EA020C7FEA645C7FEA02
:1047B000655C00F0E2804FEA5454D4EB5555B8BF25
:1047C0006D420CDD2C4480EA020281EA030382EA96
:1047D000000083EA010180EA020281EA0303362D28
:1047E00088BF30BD11F0004F4FEA01314FF4801CFB
:1047F0004CEA113102D0404261EB410113F0004F0D
:104800004FEA03334CEA133302D0524263EB4303C3
:1048100094EA050F00F0A780A4F10104D5F1200E61
:104820000DDB02FA0EFC22FA05F2801841F10001BC
:1048300003FA0EF2801843FA05F359410EE0A5F190
:1048400020050EF1200E012A03FA0EFC28BF4CF0C1
:10485000020C43FA05F3C01851EBE37101F0004577
:1048600007D54FF0000EDCF1000C7EEB00006EEB84
:104870000101B1F5801F1BD3B1F5001F0CD349080E
:104880005FEA30004FEA3C0C04F101044FEA445265
:1048900012F5800F80F09A80BCF1004F08BF5FEAEC
:1048A000500C50F1000041EB045141EA050130BDCC
:1048B0005FEA4C0C404141EB010111F4801FA4F16F
:1048C0000104E9D191F0000F04BF01460020B1FAC4
:1048D00081F308BF2033A3F10B03B3F120020CDAFC
:1048E0000C3208DD02F1140CC2F10C0201FA0CF0DA
:1048F00021FA02F10CE002F11402D8BFC2F1200C3F
:1049000001FA02F120FA0CFCDCBF41EA0C019040F4
:10491000E41AA2BF01EB0451294330BD6FEA04043D
:104920001F3C1CDA0C340EDC04F11404C4F1200228
:1049300020FA04F001FA02F340EA030021FA04F33A
:1049400045EA030130BDC4F10C04C4F1200220FA91
:1049500002F001FA04F340EA0300294630BD21FACF
:1049600004F0294630BD94F0000F83F4801306BF95
:1049700081F480110134013D4EE77FEA645C18BF89
:104980007FEA655C29D094EA050F08BF90EA020F20
:1049900005D054EA000C04BF1946104630BD91EA18
:1049A000030F1EBF0021002030BD5FEA545C05D11B
:1049B0004000494128BF41F0004130BD14F580045A
:1049C0003CBF01F5801130BD01F0004545F0FE41CE
:1049D00041F470014FF0000030BD7FEA645C1ABF03
:1049E000194610467FEA655C1CBF0B46024650EA3A
:1049F000013406BF52EA033591EA030F41F4002166
:104A000030BD00BF90F0000F04BF0021704730B5EB
:104A10004FF4806404F132044FF000054FF00001C0
:104A200050E700BF90F0000F04BF0021704730B581
:104A30004FF4806404F1320410F0004548BF404256
:104A40004FF000013EE700BF42004FEAE2014FEAAB
:104A500031014FEA02701FBF12F07F4393F07F4F86
:104A600081F06051704792F0000F14BF93F07F4FB8
:104A7000704730B54FF4607401F0004521F00041FB
:104A800020E700BF50EA010208BF704730B54FF081
:104A900000050AE050EA010208BF704730B511F086
:104AA000004502D5404261EB41014FF4806404F1BE
:104AB00032045FEA915C3FF4DCAE4FF003025FEA40
:104AC000DC0C18BF03325FEADC0C18BF033202EBC8
:104AD000DC02C2F1200300FA03FC20FA02F001FA22
:104AE00003FE40EA0E0021FA02F11444C1E600BFC1
:104AF00070B54FF0FF0C4CF4E06C1CEA11541DBF74
:104B00001CEA135594EA0C0F95EA0C0F00F0DEF83E
:104B10002C4481EA030621EA4C5123EA4C5350EA23
:104B2000013518BF52EA033541F4801143F4801374
:104B300038D0A0FB02CE4FF00005E1FB02E506F005
:104B40000042E0FB03E54FF00006E1FB03569CF05A
:104B5000000F18BF4EF0010EA4F1FF04B6F5007F60
:104B600064F5407404D25FEA4E0E6D4146EB0606D2
:104B700042EAC62141EA55514FEAC52040EA5E505B
:104B80004FEACE2EB4F1FD0C88BFBCF5E06F1ED805
:104B9000BEF1004F08BF5FEA500E50F1000041EB3C
:104BA000045170BD06F0004646EA010140EA0200E9
:104BB00081EA0301B4EB5C04C2BFD4EB0C0541EA0B
:104BC000045170BD41F480114FF0000E013C00F320
:104BD000AB8014F1360FDEBF002001F0004170BD44
:104BE000C4F10004203C35DA0C341BDC04F114045D
:104BF000C4F1200500FA05F320FA04F001FA05F2E9
:104C000040EA020001F0004221F0004110EBD370B5
:104C100021FA04F642EB06015EEA430E08BF20EAE1
:104C2000D37070BDC4F10C04C4F1200500FA04F384
:104C300020FA05F001FA04F240EA020001F0004116
:104C400010EBD37041F100015EEA430E08BF20EA89
:104C5000D37070BDC4F1200500FA05F24EEA020ED1
:104C600020FA04F301FA05F243EA020321FA04F000
:104C700001F0004121FA04F220EA020000EBD370B7
:104C80005EEA430E08BF20EAD37070BD94F0000FB7
:104C90000FD101F00046400041EB010111F4801FEB
:104CA00008BF013CF7D041EA060195F0000F18BF9C
:104CB000704703F00046520043EB030313F4801FD8
:104CC00008BF013DF7D043EA0603704794EA0C0F92
:104CD0000CEA135518BF95EA0C0F0CD050EA4106A8
:104CE00018BF52EA4306D1D181EA030101F0004125
:104CF0004FF0000070BD50EA410606BF104619464D
:104D000052EA430619D094EA0C0F02D150EA013658
:104D100013D195EA0C0F05D152EA03361CBF104699
:104D200019460AD181EA030101F0004141F0FE4138
:104D300041F470014FF0000070BD41F0FE4141F4BC
:104D4000780170BD70B54FF0FF0C4CF4E06C1CEABC
:104D500011541DBF1CEA135594EA0C0F95EA0C0F71
:104D600000F0A7F8A4EB050481EA030E52EA03352C
:104D70004FEA013100F088804FEA03334FF080554D
:104D800045EA131343EA12634FEA022245EA11157A
:104D900045EA10654FEA00260EF000419D4208BF2B
:104DA000964244F1FD0404F5407402D25B084FEAD8
:104DB0003202B61A65EB03055B084FEA32024FF484
:104DC00080104FF4002CB6EB020E75EB030E22BFE1
:104DD000B61A754640EA0C005B084FEA3202B6EBA1
:104DE000020E75EB030E22BFB61A754640EA5C0050
:104DF0005B084FEA3202B6EB020E75EB030E22BFE0
:104E0000B61A754640EA9C005B084FEA3202B6EBE0
:104E1000020E75EB030E22BFB61A754640EADC009F
:104E200055EA060E18D04FEA051545EA16754FEA01
:104E300006164FEAC30343EA52734FEAC2025FEA1F
:104E40001C1CC0D111F4801F0BD141EA00014FF0AE
:104E500000004FF0004CB6E711F4801F04BF01437F
:104E60000020B4F1FD0C88BFBCF5E06F3FF6AFAE9B
:104E7000B5EB030C04BFB6EB020C5FEA500C50F12B
:104E8000000041EB045170BD0EF0004E4EEA1131AE
:104E900014EB5C04C2BFD4EB0C0541EA045170BDB5
:104EA00041F480114FF0000E013C90E645EA060EF9
:104EB0008DE60CEA135594EA0C0F08BF95EA0C0F27
:104EC0003FF43BAF94EA0C0F0AD150EA01347FF46F
:104ED00034AF95EA0C0F7FF425AF104619462CE746
:104EE00095EA0C0F06D152EA03353FF4FDAE1046A9
:104EF000194622E750EA410618BF52EA43067FF4FA
:104F0000C5AE50EA41047FF40DAF52EA43057FF489
:104F1000EBAE12E74FEA410212F5001215D211D59D
:104F20006FF47873B3EB625212D94FEAC12343F0A6
:104F3000004343EA505311F0004F23FA02F018BF28
:104F4000404270474FF00000704750EA013005D1F1
:104F500011F0004008BF6FF0004070474FF00000B4
:104F6000704700BF4FEA4102B2F1E04324BFB3F5FE
:104F7000001CDCF1FE5C0DD901F0004C4FEAC002D0
:104F80004CEA5070B2F1004F40EB830008BF20F0B4
:104F90000100704711F0804F21D113F13872BCBF6E
:104FA00001F00040704741F480114FEA5252C2F1C3
:104FB0001802C2F1200C10FA0CF320FA02F018BF0C
:104FC00040F001004FEAC1234FEAD32303FA0CFC5F
:104FD00040EA0C0023FA02F34FEA4303CCE77FEAEE
:104FE000625307D150EA01331EBF4FF0FE4040F438
:104FF0004000704701F0004040F0FE4040F40000E7
:10500000704700BF80F0004002E000BF81F0004127
:1050100042001FBF5FEA410392EA030F7FEA226C5E
:105020007FEA236C6AD04FEA1262D2EB1363C1BFEE
:10503000D218414048404140B8BF5B42192B88BF5D
:10504000704710F0004F40F4000020F07F4018BF80
:10505000404211F0004F41F4000121F07F4118BFA0
:10506000494292EA030F3FD0A2F1010241FA03FC48
:1050700010EB0C00C3F1200301FA03F100F0004330
:1050800002D5494260EB4000B0F5000F13D3B0F1F8
:10509000807F06D340084FEA310102F10102FE2A67
:1050A00051D2B1F1004F40EBC25008BF20F00100D7
:1050B00040EA03007047490040EB000010F4000F85
:1050C000A2F10102EDD1B0FA80FCACF1080CB2EB18
:1050D0000C0200FA0CF0AABF00EBC2505242184377
:1050E000BCBFD0401843704792F0000F81F400011C
:1050F00006BF80F400000132013BB5E74FEA4103EF
:105100007FEA226C18BF7FEA236C21D092EA030F5A
:1051100004D092F0000F08BF0846704790EA010FD4
:105120001CBF0020704712F07F4F04D1400028BF01
:1051300040F00040704712F100723CBF00F50000E3
:10514000704700F0004343F0FE4040F40000704719
:105150007FEA226216BF08467FEA236301464202C5
:1051600006BF5FEA412390EA010F40F480007047D8
:105170004FF0000304E000BF10F0004348BF40427E
:105180005FEA000C08BF704743F0964301464FF0BA
:1051900000001CE050EA010208BF70474FF0000316
:1051A0000AE000BF50EA010208BF704711F0004357
:1051B00002D5404261EB41015FEA010C02BF844627
:1051C0000146002043F0B64308BFA3F18053A3F586
:1051D0000003BCFA8CF2083AA3EBC25310DB01FACD
:1051E00002FC634400FA02FCC2F12002BCF1004F51
:1051F00020FA02F243EB020008BF20F001007047E2
:1052000002F1200201FA02FCC2F1200250EA4C0035
:1052100021FA02F243EB020008BF20EADC7070477B
:105220004FF0FF0C1CEAD0521EBF1CEAD15392EA89
:105230000C0F93EA0C0F6FD01A4480EA010C400265
:1052400018BF5FEA41211ED04FF0006343EA5010BF
:1052500043EA5111A0FB01310CF00040B1F5000F01
:105260003EBF490041EAD3715B0040EA010062F1B0
:105270007F02FD2A1DD8B3F1004F40EBC25008BF9A
:1052800020F00100704790F0000F0CF0004C08BFB8
:1052900049024CEA502040EA51207F3AC2BFD2F185
:1052A000FF0340EAC250704740F400004FF0000393
:1052B000013A5DDC12F1190FDCBF00F000407047CD
:1052C000C2F10002410021FA02F1C2F1200200FA0B
:1052D00002FC5FEA310040F1000053EA4C0308BFD2
:1052E00020EADC70704792F0000F00F0004C02BF23
:1052F000400010F4000F013AF9D040EA0C0093F09E
:10530000000F01F0004C02BF490011F4000F013BF7
:10531000F9D041EA0C018FE70CEAD15392EA0C0F65
:1053200018BF93EA0C0F0AD030F0004C18BF31F0D0
:10533000004CD8D180EA010000F00040704790F0A6
:10534000000F17BF90F0004F084691F0000F91F04A
:10535000004F14D092EA0C0F01D142020FD193EA10
:105360000C0F03D14B0218BF084608D180EA010098
:1053700000F0004040F0FE4040F40000704740F074
:10538000FE4040F4400070474FF0FF0C1CEAD05242
:105390001EBF1CEAD15392EA0C0F93EA0C0F69D09E
:1053A000A2EB030280EA010C49024FEA402037D009
:1053B0004FF0805343EA111143EA10130CF0004000
:1053C0008B4238BF5B0042F17D024FF4000C8B42F0
:1053D00024BF5B1A40EA0C00B3EB510F24BFA3EBD0
:1053E000510340EA5C00B3EB910F24BFA3EB9103A0
:1053F00040EA9C00B3EBD10F24BFA3EBD10340EAFA
:10540000DC001B0118BF5FEA1C1CE0D1FD2A3FF63F
:1054100050AF8B4240EBC25008BF20F001007047F4
:105420000CF0004C4CEA50207F32C2BFD2F1FF0397
:1054300040EAC250704740F400004FF00003013AC8
:1054400037E792F0000F00F0004C02BF400010F46C
:10545000000F013AF9D040EA0C0093F0000F01F080
:10546000004C02BF490011F4000F013BF9D041EAA2
:105470000C0195E70CEAD15392EA0C0F08D14202D5
:105480007FF47DAF93EA0C0F7FF470AF084676E7A8
:1054900093EA0C0F04D14B023FF44CAF08466EE781
:1054A00030F0004C18BF31F0004CCAD130F000424F
:1054B0007FF45CAF31F000437FF43CAF5FE700BFA7
:1054C0004FF0FF3C06E000BF4FF0010C02E000BFD0
:1054D0004FF0010C4DF804CD4FEA40024FEA410372
:1054E0007FEA226C18BF7FEA236C11D001B052EA28
:1054F000530C18BF90EA010F58BFB2EB030088BFEE
:10550000C81738BF6FEAE17018BF40F0010070475C
:105510007FEA226C02D15FEA402C05D17FEA236C3E
:10552000E4D15FEA412CE1D05DF8040B704700BF85
:10553000844608466146FFE70FB5FFF7C9FF00281C
:1055400048BF10F1000F0FBD4DF808EDFFF7F4FF55
:105550000CBF012000205DF808FB00BF4DF808EDEE
:10556000FFF7EAFF34BF012000205DF808FB00BF11
:105570004DF808EDFFF7E0FF94BF012000205DF833
:1055800008FB00BF4DF808EDFFF7D2FF94BF0120E4
:1055900000205DF808FB00BF4DF808EDFFF7C8FFDD
:1055A00034BF012000205DF808FB00BF4FEA400235
:1055B000B2F1FE4F0FD34FF09E03B3EB12620DD941
:1055C0004FEA002343F0004310F0004F23FA02F0AB
:1055D00018BF404270474FF00000704712F1610F52
:1055E00001D1420205D110F0004008BF6FF0004029
:1055F00070474FF00000704742000ED2B2F1FE4FEC
:105600000BD34FF09E03B3EB126209D44FEA002391
:1056100043F0004323FA02F070474FF00000704758
:1056200012F1610F01D1420202D14FF0FF307047F9
:105630004FF00000704700BF03685A004CBF43F0B2
:10564000004323F000431844704700BF61B32DE9C5
:10565000F84F01F1FF3A90460646D146002707EB86
:10566000090404EBD4746410E50071190846FFF7CF
:10567000E3FFA245834605F10800304409D0FFF757
:10568000DBFFC34500F1FF3005D8404509D2671C58
:10569000E5E7C34505D9A74202D004F1FF39DEE7AB
:1056A00000210846BDE8F88F08467047012807D05A
:1056B000022807D0044B00280CBF18460020704772
:1056C0000248704702487047C15D0008C55D000888
:1056D000C95D000830B5254B83B004468D1E7BB3F1
:1056E00001A92846AFF3008020B301992A46FFF7AD
:1056F000ADFF0146F0B1FFF79FFF4B68A064012B9F
:1057000012D0002B01F1040021DBFFF795FF0023ED
:10571000E06423650368002B1DDBFFF78DFF00238A
:105720002061184603B030BD0023236105231846CD
:1057300003B030BD002323610923184603B030BDF8
:105740000B490C4B0846591AC9100191CEE70123A9
:10575000E0642365DEE7C3F30360FFF7A7FF0028DB
:10576000206114BF00230923DBE700BF0000000015
:1057700018A0000850A10008036810B5DA07044615
:1057800006D49B0700F1480009D500F05BFC2368B4
:10579000590709D51A070ED5DB0613D510BD00F041
:1057A00049FC23685907F5D404F1D00000F052FCFD
:1057B00023681A07F0D404F5A87000F053FC23689E
:1057C000DB06EBD404F5E870BDE8104000F08EBCB9
:1057D00003680BB11844704718467047092070479A
:1057E000704700BF70B504460D4608E02A6C236977
:1057F000626121462A4601209847082808D1296C71
:105800002046FFF767FF06460028EFD0FEF766FA4E
:105810000728FBD13046296CFFF7E2FF281D00F076
:10582000FDFB00BF2DE9F0470646ADF5727D03ADE7
:105830000C1D17460FCC0FC50FCC0FC50FCC0FC5D5
:1058400094E80F0002ACD6F80C80D6F8189085E8E2
:105850000F0000233046216C2360FFF73BFF054615
:10586000002F14BF0A2709277DB1A36B47F0100151
:105870008DE810023246636401203346C04778BB8E
:1058800028460DF5727DBDE8F087236C4FF4F07269
:10589000736121467AA800F075FE33697AAA314611
:1058A00038469847889B82468DE8100239466364E3
:1058B000324633460120C04790B94FF4F0727AA9BE
:1058C000204600F05FFEBAF1080F06D1216C304689
:1058D000FFF700FF09270546C6E7BAF1070F04D016
:1058E00009200DF5727DBDE8F0872846216CFFF791
:1058F00077FF03A800F092FB406C7047F0B5CB6BCC
:10590000F9B00B640E1D01AD0F4604460FCE0FC556
:105910000FCE0FC50FCE0FC596E80F004FF0FF3624
:1059200085E80F00009606E023696A4621469847FD
:105930000828054608D110992046FFF7CBFE00281D
:10594000F2D0092079B0F0BD6846FFF715FF062DAB
:10595000F7D139462046FFF745FF00BF30B4DD6B75
:10596000C160826119461D64002230BC5AE700BF45
:1059700070B54369C6680B6426B10122FFF752FF78
:10598000FEF7ACF903690A4604460D4601460220BB
:105990009847072807D0082803D129462046FFF753
:1059A00021FFFEF79BF93046296CFFF719FF281DF0
:1059B00000F034FBC2682AB110B4CC6B00220C6436
:1059C00010BC2FE79AE700BF704700BF836813B190
:1059D000014601201847704700B5042907D8DFE8C1
:1059E00001F00309060909000BB90F2A05D90220A5
:1059F0005DF804FB01205DF804FB00EB82025268B5
:105A00001846019B1A605DF804FB00BF10B584B016
:105A1000002303AC0A4600941946FFF7DDFF039804
:105A200004B010BD00B5042907D8DFE801F0030970
:105A3000060909000BB90F2A05D902205DF804FBFD
:105A400001205DF804FB019900EB82020968184609
:105A500051605DF804FB00BF10B584B004AC44F89D
:105A6000042D00230A4600941946FFF7DBFF04B01B
:105A700010BD00BFF0B5D36BADF50F7D1364151DE0
:105A800017AC07460E460FCD0FC40FCD0FC40FCD78
:105A90000FC495E80F004FF0FF3584E80F0016950E
:105AA00011E016A86A46FFF7D7FF314616A8B84797
:105AB00080B9049B16AA6946082098470528044621
:105AC00009D0092806D026996846FFF703FE0C2165
:105AD0000028E6D0092416A8FFF74EFE20460DF553
:105AE0000F7DF0BD2DE9F04FCC6C914622688BB054
:105AF00004340D460792089400F0030B1E46002B59
:105B000064D11202032307928DF825608DF82430AA
:105B10002B6DBBF1020F08BFAC6B13F0010343D137
:105B200000F00800C2B2039201932768002F3DD015
:105B3000022E47D02788B4F802800434AB6C28F0DA
:105B4000010A0F2148469A44FFF760FF824537D883
:105B500027F001039A4450452CBF002001204FEA52
:105B6000480808F0020807F0010748EA0708B8F1FA
:105B7000010F41D038D3B8F1020F1DD1236823F0B3
:105B800000420292BBF1000F79D130B10399002994
:105B900000F08180002A00F0A880002B79DB029BB6
:105BA000013304EB8304C0E700230193022E40DDA0
:105BB000FFF714FE002842D009200BB0BDE8F08F9B
:105BC0000020CCE7D4F804800834B7E7022B9FDC30
:105BD000130CD9B212048DF82530022304EB810492
:105BE00007928DF8243093E7BBF1000F02D0002814
:105BF00040F0B080043498E7BBF1000F26D1B0B17B
:105C000094E80C00991C4FEAD272D5D005F15801E6
:105C10000133069100F09480201DFFF7D9FD06ABFB
:105C200001462846AFF30080002840F0B8800834D1
:105C30007BE707A9484600F0F3FA0028BCD1019B96
:105C4000002B5CD108200BB0BDE8F08F0D21484639
:105C50002F6AFFF7DBFE8742E9D1AB6A9C42E6D1AF
:105C60002046FFF7E9FC0F2102464846FFF7F4FE05
:105C700048462A460021FFF7EFFE07209DE70D2149
:105C800048462F6AFFF7C2FE874248D02368002BA0
:105C900085DA043483E7029B3BB305F15803271DE3
:105CA000CDF810B0DDF80C80A346DDF808A01C4646
:105CB000059602E0B245B04616D038460694FFF786
:105CC00087FD06AB014600222846AFF3008008F1AD
:105CD000010604370028EDD0029B5C464345DDF801
:105CE00010B0059ED2D100E05C4648460D21FFF77A
:105CF0008DFE069B2862AC626B6206205DE70F2179
:105D00004846FFF783FE0E2102464846FFF7A4FEF1
:105D100048462A4A0F21FFF79FFE07204DE7AB6A4E
:105D20009C42B3D1042202990027A318A962EF6212
:105D30002A636B632368BB421FDB012301932EE7B9
:105D400048460D21FFF762FE2862069B6B62AC623B
:105D5000062032E72046FFF76FFC04340646AC63AA
:105D60002846AFF3008000283FF426AF484632466D
:105D70000F21FFF771FE07201FE70846013004EBF3
:105D80008000FFF759FC0F2102464846FFF764FEEA
:105D900048462A463946FFF75FFE07200DE70746CB
:105DA0000D214846FFF732FE022F2862CDD12B4647
:105DB000069A43F82C2F6B62C9E700BF0000000071
:105DC00000238FE601238DE602238BE6F0B504461F
:105DD000C5B004290DD8DFE801F057030C310F00DE
:105DE000012B4FEA124695B266D17219102A40F281
:105DF0009F80022045B0F0BD002BFAD1102AF8D8C0
:105E00002368D80600F1C98022AE3046019200F026
:105E100077F9A06B019A0023012505FA03F11142DD
:105E200003D00168043046F823100133042BF4D169
:105E3000A063304600F05AF90020DBE7032BD8D1ED
:105E4000150C97B2EB19102BD3D823681E0700F15D
:105E5000B88022AE30467F0000F026F906EBC5027E
:105E60007B1EA56B57B12946043A51F8040B013B40
:105E700042F8040F581CF8D105EB87053046A5639E
:105E800000F0F0F80020B5E7002BB2D1A56B97B277
:105E9000201D012606FA03F1394203F1010302D065
:105EA000296804350160102B00F10400F2D112F4CE
:105EB00000503BD1A5639DE7052B9AD17719202F80
:105EC00097D80F2E65D92F46002D48D12A46002796
:105ED000002AA06B71DD00EBC202014644A800EB72
:105EE000C6008C3851F8045B914240F8045FF9D148
:105EF000084697B13246102E44A938BF102201EB54
:105F0000C202A2F5C4727900043A00EB810150F894
:105F1000045B814242F8045FF9D1012B47D00F2E78
:105F2000A16332D917B102A800F094F8002061E70C
:105F30000F2E3FF65EAF00272268D1070DD522F065
:105F40000101052B21600193204652D022F003026B
:105F500040F8482B00F072F8019B002F51D02268C6
:105F6000510736D4012B3ED00F2E06D822A801931C
:105F700000F06CF8019B002FA8D002A8019300F05C
:105F80006DF8019BC6F11002A2E722A800F05AF8B2
:105F9000C8E7102FCFD9103FCEE723F010032360BE
:105FA00004F5E870019200F0ABF8019A2CE7043197
:105FB000A16322A800F03EF8B8E7002F9AD101466D
:105FC000ABE723F00803236004F5A87000F06CF839
:105FD0003FE7204622F0040240F8D02B019300F066
:105FE0003DF8019BBEE722A8019300F027F8019B32
:105FF000C8E741F0020140F8481B00F027F8019B78
:10600000ABE7012B03D00F2E3FF660AFAEE722A81F
:10601000019300F013F8019B58E700BF00F1340131
:1060200091E838009C46A6464CF8045D90E8FF0FC6
:10603000E54600BD90EC210B704700BF80EC210BC2
:10604000704700BF90EC200B704700BF80EC200B26
:10605000704700BFD0EC200B704700BFC0EC200B96
:10606000704700BFF0EC0201F0EC0211F0EC0221ED
:10607000F0EC0231F0EC0241F0EC0251F0EC026184
:10608000F0EC0271F0EC0281F0EC0291F0EC02A174
:10609000F0EC02B1F0EC02C1F0EC02D1F0EC02E164
:1060A000F0EC02F1704700BFE0EC0201E0EC0211FD
:1060B000E0EC0221E0EC0231E0EC0241E0EC0251C4
:1060C000E0EC0261E0EC0271E0EC0281E0EC0291B4
:1060D000E0EC02A1E0EC02B1E0EC02C1E0EC02D1A4
:1060E000E0EC02E1E0EC02F1704700BFB0FC01819E
:1060F000B0FC0191B0FC01A1B0FC01B1704700BF40
:10610000A0FC0181A0FC0191A0FC01A1A0FC01B1B7
:10611000704700BFEC4600B52DE900502DE9FF1F88
:106120004FF000032DE90C0001A9FFF7E7FBDDF8B4
:1061300040E012B0704700BFEC4600B52DE90050BA
:106140002DE9FF1F4FF000032DE90C0001A9FFF717
:106150000FFCDDF840E012B0704700BFEC4600B520
:106160002DE900502DE9FF1F4FF000032DE90C0031
:1061700001A9FFF71FFCDDF840E012B0704700BF37
:10618000EC4600B52DE900502DE9FF1F4FF000034C
:106190002DE90C0001ABFFF7E1FBDDF840E012B0A8
:1061A000704700BFEC4600B52DE900502DE9FF1FF8
:1061B0004FF000032DE90C0001AAFFF75BFCDDF8AE
:1061C00040E012B0704700BF037A1BB9437A43B96D
:1061D000B02070475A1E036802721A020260180E3D
:1061E00070474268013B10B4437213680321141DC9
:1061F00001721A024460026010BC180E704700BFA2
:1062000000B585B003AA0023009219460C22FFF7BF
:10621000E3FB039805B05DF804FB00BFF0E700BFA7
:106220002DE9F04306460D4685B04FF0000828469C
:10623000FFF7CAFFB028044600F0B48020F07F03C7
:1062400013F0FF0320D000F0F003802B7AD0902BC6
:1062500035D0A02B48D0B02B5CD0C02B00F089806B
:1062600000F0F803D02B0BD100F00702013242F40A
:106270000022052301213046FFF7A8FD0028D6D0D3
:10628000092005B0BDE8F0830DF10C09194687001F
:10629000CDF800900D223046FFF79EFBFFB2039B26
:1062A000043760064CBFDF1BFF180023CDF80090B9
:1062B00019460D2230460397FFF7B4FBB7E700F00D
:1062C0000D030D2BDCD003AF002300F00F021946A5
:1062D00000973046FFF780FB0023009719460D22F8
:1062E0003046FFF79FFBA2E7C2434FF47F6302F003
:1062F000070243FA02F2010702EA03024FF0000329
:1063000048BF42F4804219463046FFF75FFD00283F
:10631000B6D18CE7B1284AD0B22853D0B32800F0C8
:10632000818000F0FC03B42BAAD000F007020132F8
:10633000012342F4002219463046FFF747FD0028AA
:106340009ED174E72846FFF73FFF24022043B0F5B3
:10635000004F95D004010023A2B219463046FFF742
:1063600035FD00288CD114F4004F18BF4FF0010800
:106370005DE7C62862D0C7286CD000F0F803C02BB8
:106380007BD0C82800F09180C9287FF479AF2846D7
:10639000FFF71AFF020300F00F0002F47022013031
:1063A000024366E7B8F1000F6ED0002069E7284687
:1063B000FFF70AFF024600283FF462AF10F0F00337
:1063C000B9D05DE700230DF10C090D221946CDF877
:1063D00000903046FFF700FB2846FFF7F5FE020667
:1063E0004FF002040CD5039B00F07F00A040034453
:1063F00028460393FFF7E8FE030604F10704F2D4EE
:10640000039B00F07F0000FA04F203F501740023FF
:106410001444CDF8009019460D2230460394FFF73E
:1064200001FB04E72846FFF7CFFE010300F00F0051
:1064300001F47021421C01230A437CE72846FFF740
:10644000C3FE010300F00F0001F47021421C03237E
:106450000A4370E72846FFF7B7FE024600283FF4DC
:106460000FAF10F0F0037FF40BAF04213046FFF7BD
:10647000ADFC00287FF404AFD9E600F00F02013232
:10648000032342F4202256E703AC43460E22414642
:1064900000943046FFF7A0FA0094304643460F229E
:1064A0004146FFF7BFFA4046EBE62846FFF78CFE71
:1064B00000F0F00200F00F031032013343EA023221
:1064C000D7E600BF10B5C36C84B003205A688DF8BE
:1064D0000C00DC7912020833084601A901928DF8FC
:1064E0000D400293FFF79CFE04B010BD08B5FFF706
:1064F00095FE806C08BD00BF08B5FFF78FFEC36C2A
:10650000D87903EB8000083008BD00BF08B5FDF75F
:10651000E5FB00BF08B5FFF7F9FF00BF002100F061
:10652000C3BE0A22002100F059BF0000034B1B68C4
:10653000186A034B002808BF18467047F002002075
:1065400024010020D0F8EC007047000008B5034B90
:106550001868FFF7EBFFD0F8EC0008BDF002002050
:1065600082B001B901A93AB143B113780B60127836
:10657000101C18BF012003E0104601E06FF001007D
:1065800002B0704710B5431E0A44914204D011F87E
:10659000014B03F8014FF8E710BD03460244934254
:1065A00002D003F8011BFAE7704700000EB400B5F3
:1065B0004FF402719CB0ADF814106FF000410491DB
:1065C00007914FF6FF711DAB02900690084853F8F3
:1065D000042BADF81610006802A9019301F0F0FE3B
:1065E000029B00221A701CB05DF804EB03B07047E8
:1065F000F0020020F8B506460F4616F8014BFFF7EB
:10660000A5FF2044437817F8015B03F00303012B37
:1066100008BF2034FFF79AFF2844437803F00303B0
:10662000012B14BF2B4605F12003E01A01D1002BEA
:10663000E3D1F8BD034611F8012B03F8012B002A22
:10664000F9D17047034613F8012B002AFBD1181A21
:1066500001387047034610B542B111F8014B013AB9
:1066600003F8014B002CF7D11A4400E010BD93420F
:1066700002D003F8014BFAE710BD2DE9F0410F46B7
:10668000904601F0B3FC04460D46B8F1000F11D05E
:10669000C7F30A53C3F16B03002B0BDD1B0503F19A
:1066A0007F55002405F5401522462B46FEF720FABB
:1066B000BDE8F08120462946BDE8F08100000000D9
:1066C0002DE9F04F1F469FB00023824638461A93AB
:1066D0000691159201F0C3F906460068FFF7B2FF74
:1066E0000446069B4FF000084FF000091993199BD0
:1066F0001A780D2A05D8092A13D2002A00F09681AB
:1067000011E02B2A04D02D2A04D0202A0BD108E036
:10671000002200E001220E925A1C19925B7823B9E4
:1067200084E10133E2E700230E93199D2B78302B8F
:106730005DD16B78582B01D0782B4DD10E9B0297F1
:1067400001931AAB00939E4A1BAB19A9504600F067
:10675000B3FE10F00706044600F07185062E05D141
:106760000135002319950E9300F069BD1A9A3AB1CC
:1067700035211CA801F021FD1A99504601F0A6F917
:10678000062E22D8DFE806F0040D08181D0D0400BF
:106790004FF00009C84618E0DDF87080DDF874900D
:1067A00013E01D9B1B9A23F4801302F23342DDF8A1
:1067B000708043EA025908E0DFF808924FF00008C1
:1067C00003E06FF000494FF0FF38210740F13785B3
:1067D00049F0004900F033BD199B5A1C19925B78AF
:1067E000302BF9D0002B00F02A85012300E0002394
:1067F0000893199B0A22099300239B46059304934F
:1068000019980578A5F13003D9B209290ED8049951
:1068100001300829C9BF059902FB0B3B02FB01337C
:106820000593049B199001330493E9E722463168EC
:1068300002F066F828B100202B460246049D01466E
:106840004DE0199B1A191992049A1B5D002A3FD139
:106850001046302B05D1199B01305A1C19925B78D8
:10686000F7E7A3F13102082A3FD8199A09920246A4
:1068700000200546303B00F1010123D00A4429469F
:106880002E180A24B1420CD001314F1E082F02DC11
:1068900004FB0BFBF6E71029DEBF059F6743059756
:1068A000F0E72844082800F1010503DC0A2101FB78
:1068B0000B3B06E0102DDFBF05980A2101FB0033DA
:1068C00005930021199B581C19905B78084601E03C
:1068D0000246049DA3F130010929CBD90121652B82
:1068E00001D0452B54D16DB904E0652B40F0B5843F
:1068F0000022012128B9089B002B00F09780054653
:1069000000E00025199B069301331993069B5B78E1
:106910002B2B06D02D2B02D00024079408E0012356
:1069200000E000230793069B02331993069B9B7894
:10693000A3F13004092C29D8302B04D1199B5C1CFD
:1069400019945B78F8E7A3F13104082C20D8A3F15F
:106950003007199B4FF00A0E1E46199B5C1C1994B8
:106960005B78A3F1300CBCF1090F03D80EFB07379D
:10697000303FF2E7A41B082C44F61F6402DCBC4243
:10698000A8BF3C46079E26B1644202E0069C1994CB
:106990000024002D54D1002840F05184089A002A88
:1069A00040F04D84002941D14E2B20D002DC492BF0
:1069B0000AD03BE0692B07D06E2B18D036E000BF21
:1069C000989D00080000F07FAB4919A800F0A6FFD1
:1069D00060B3199BA949013B19A8199300F09EFFC8
:1069E00010B9199B01331993DFF8AC921AE0A4494E
:1069F00019A800F093FFC8B1199B1B78282B0FD161
:106A00001CAAA04919A800F09CFF052808D11D9BCD
:106A1000DDF8708043F0FF4949F4E00900F00FBC55
:106A2000DFF878924FF0000800F009BC069B19933C
:106A3000159B002B00F00E8400230E9300F001BC88
:106A4000049BA71A002B08BF2B462C46102D584636
:106A5000A8BF10240493FDF7D5FF092C8046894672
:106A600013DD894B03EBC40353E91223FEF740F80F
:106A7000804605988946FDF7C5FF02460B4640460D
:106A80004946FDF783FE804689460F2D33DC002FF3
:106A900000F0D58322DD162F07DC7B4D424605EB47
:106AA000C7014B46D1E9000113E0C5F125039F4220
:106AB00021DC754CC5F10F0504EBC5017D1B424679
:106AC000D1E900014B4604EBC504FEF711F8D4E907
:106AD0000023FEF70DF880468946B0E317F1160F44
:106AE00009DB694D4046A5EBC703D3E900234946BE
:106AF000FEF728F9EFE72C1B3C44002C5DDD14F079
:106B00000F010AD0604B424603EBC101D1E90001FD
:106B10004B46FDF7EDFF8046894634F00F0400F048
:106B2000C180B4F59A7F0FDD4FF0000BCDF810B0A7
:106B3000CDF81CB0CDF818B02223CAF80030DFF829
:106B400058914FF0000889E14046494600234F4ED6
:106B500024110593012C0CDDE20704D5D6E90023AE
:106B6000FDF7C6FF0123059A64100132059208362D
:106B7000F0E70BB180468946444B059AA9F1547958
:106B800003EBC201D1E9000142464B46FDF7B0FFDD
:106B900021F0004389460A461B0D3D491B058B42E7
:106BA0008046C1D8A1F580118B4286BFDFF8F090F6
:106BB0004FF0FF3802F1547974E073D0644214F05E
:106BC0000F020AD0304B404603EBC2034946D3E9DB
:106BD0000023FEF7B7F880468946241162D01F2CA7
:106BE00008DD4FF0000BCDF810B0CDF81CB0CDF89B
:106BF00018B02CE14046494614F0100F0CBF00239A
:106C00006A23244E05930023002C09DDE20704D5F6
:106C1000D6E90023FDF76CFF012364100836F3E783
:106C20000BB180468946059BEBB1C9F30A53C3F10A
:106C30006B03002B494616DD1F2B0EDD342BDEBF08
:106C4000203B4FF0FF3202FA03F34FF00008CCBFB5
:106C50004FF05C7903EA010905E04FF0FF3202FAD8
:106C600003F303EA0808002200234046494601F0E6
:106C700063FF0028B5D117E0AC9D0008AF9D000868
:106C8000B59D0008B89D0008D09E0008989F000898
:106C90000000A07C709D00080000F07F0000F8FF5D
:106CA000FFFFEF7F00230593CDF800B02B46049A39
:106CB0000999504600F05CFF079000283FF434AF7C
:106CC000002FC7F10003A8BF00230F934FF0000B64
:106CD00027EAE7731493CDF810B0079B5046596824
:106CE00000F0BFFE069000283FF426AF079B0C3053
:106CF0001A6903F10C0102329200FFF743FC1CAB4E
:106D000001931BAB009342464B465046CDE90A899E
:106D100001F0DDF91A9000283FF40EAF0121504632
:106D200000F0B1FF049000283FF406AF1B9B0599CB
:106D3000002BACBF0F9A149A1C9CACBFD618D21A69
:106D4000A3EB01032344B14903F1FF33ACBF149A11
:106D50000F9E8B42C4F1360480F28580C91A1F2928
:106D6000C8BFAB4D4FF00107D4BF07FA01F3ED1ACE
:106D7000A4EB0104D9BF0993002507FA05F509978B
:106D80003719059BBE4214441C443346A8BF3B46FA
:106D9000A342A8BF2346002BC2BFFF1AE41AF61A6B
:106DA0000F9B002B63D1002F7ADC149B002B40F04B
:106DB0008180002C00F38880002E00F38F80069ADB
:106DC0001A99504601F0B3F8834600283FF4B4AE58
:106DD000C3680024C4600499089301F08CF8A042B1
:106DE00080F28B80089B002B40F00282B8F1000FEC
:106DF00040F0FE81C9F31303002B40F0F98129F024
:106E000000431B0D1B05B3F1D66F40F2F181DBF897
:106E10001430002B6CD059460122504601F01AF86C
:106E20000499834601F067F8002840F3E18129F0D6
:106E30000043059A1B0D1B05002A00F08D80B3F15D
:106E4000D66F00F38980B3F15C7F00F3D3812223F6
:106E50004FF000084FF00009CAF80030079B002BE4
:106E600040F0D981EBE101230025099388E71A4618
:106E70000499504600F0A0FF049000283FF45CAE57
:106E800001461A9A504600F007FF089000283FF488
:106E900053AE1A99504600F019FE089B1A9382E7E8
:106EA0003A461A99504600F0D5FF1A9000287FF410
:106EB0007CAF41E6149A0699504600F07DFF06909B
:106EC00000287FF476AF37E622460699504600F058
:106ED000C1FF069000287FF46FAF2DE6324604997B
:106EE000504600F0B7FF049000287FF468AF23E617
:106EF000DBF81030012B8EDC7AE161D1089AC9F3FE
:106F0000130322B343494A468B422ED1059B414687
:106F100063B1414B1340B3F1D46F07D81B0DC3F1DC
:106F20006B034FF0FF3000FA03F301E04FF0FF3343
:106F30008B421AD139498A4202D101333FF4FCAD68
:106F4000354B4FF00008134003F5801950E163B949
:106F5000B8F1000F09D16AE7A3F580136FEA13595E
:106F60004FF0FF386FEA095942E115B115EA090FF0
:106F700002E0099B13EA080F00F03A81089B059A8A
:106F80004046494653B1FFF778FB02460B46DDE920
:106F90000A01FDF7FBFB8046894629E1FFF76DFBFF
:106FA00002460B46DDE90A01FDF7EEFB0022002355
:106FB0008046894601F0C0FD00287FF448AF17E104
:106FC0000499584601F0D1F800224FF0804306465C
:106FD0000F4601F0C5FD00283FD0089B13B10026E5
:106FE0000F4F10E0B8F1000F03D1C9F313033BB901
:106FF0001AE0B8F1010F03D1B9F1000F3FF427AF48
:10700000084F00260024064D3CE000BF02FCFFFFB5
:10701000E2FBFFFFFFFF0F000000F07FFFFFEF7FAD
:107020000000F03F0000F0BF0022994B3046394687
:1070300001F08CFD40B90022964B30463946FDF7F1
:1070400057FD04460D4601E0089C924D05F10043B2
:1070500016941793DDE9166714E08E4B0022304634
:107060003946FDF745FD089B04460D4623B901F15D
:1070700000431090119303E002460B46CDE9102324
:10708000DDE9106729F000431B0D1B050993099AE0
:10709000814B9A422BD1DDE90A23A9F1547940466C
:1070A0004946CDE90C2300F0A1FF02460B463046CD
:1070B0003946FDF71DFD42464B46FDF767FB21F0C3
:1070C00000431B0D754A1B05934280460CD9744B37
:1070D0000D9A9A4203D10C9B01333FF42DADDFF89A
:1070E000C0914FF0FF3872E001F1547939E0059B0F
:1070F0003BB3099BB3F1D46F23D85DA3D3E900233D
:107100002046294601F02CFDB8B12946204601F061
:1071100045FD002808BF0120FDF774FC089B0446CC
:107120000D4623B901F100431290139303E0024688
:107130000B46CDE91223DDE91267099A07F1D66300
:107140009F1ADDE90A0100F051FF02460B46304666
:107150003946FDF7CDFCDDE90A23FDF717FB804634
:107160008946059B9BBB29F000431B0D099A1B0513
:107170009A424E462BD129462046FDF7CBFEFDF71D
:1071800051FC0B46024629462046FDF7FDFA089BB6
:1071900004460D462BB9B8F1000F02D1C9F313060E
:1071A0007EB135A3D3E900232046294601F0CEFC69
:1071B00088BB33A3D3E900232046294601F0E4FC31
:1071C00004E031A3D3E9002301F0C0FC18BB1A99F5
:1071D000504600F07BFC0699504600F077FC04997D
:1071E000504600F073FC5946504600F06FFC74E5C1
:1071F000059B83B12B4B40460D9300230C934946CE
:10720000DDE90C23FDF774FC8046894619B910B9F5
:107210002223CAF800301A99504600F057FC06990C
:10722000504600F053FC0499504600F04FFC07997B
:10723000504600F04BFC5946504600F047FC159B69
:1072400013B1199B159A13600E9B1BB1424609F1AD
:10725000004307E042464B4604E000252A46012150
:10726000FFF73FBB104619461FB0BDE8F08F00BFC7
:107270000000C0FFFFFFDF419535A094FFFFDF3F17
:1072800035E5AF350000E03F9535A094FFFFCF3FD7
:107290000000F03F0000E03F0000E07FFFFF9F7C28
:1072A000FFFFEF7F00005039064B10B41C68064A00
:1072B000236A002B08BF13460A460146204610BC2D
:1072C000FFF7FEB9F0020020240100202DE9F0476D
:1072D0008046894692461E460F463D46089815F858
:1072E000014BFFF72FF92044427802F0080202F028
:1072F000FF030AB12F46F0E72D2C03D1BD1C7C788B
:10730000012303E02B2C04BF7C78BD1C16B1102E8A
:107310000AD15EE0302C5AD12A7802F0DF02582AD6
:1073200050D16C7810260235002B14BF4FF000426C
:107330006FF00042B2FBF6FE06FB1E210022104653
:10734000A4F13007092F01D83C460AE0A4F1410717
:10735000192F01D8373C04E0A4F16107192F13D885
:10736000573CA64210DD571C0BD0864507D301D1F0
:10737000A14203DB00FB0640012202E070464FF011
:10738000FF3215F8014BDBE7511C0ED1002B4FF0FB
:10739000220314BF4FF000406FF00040C8F80030E7
:1073A000BAF1000F07D1BDE8F08703B14042BAF14E
:1073B000000F11D00AB1013D00E04D46CAF800505F
:1073C000BDE8F0873024002EAED10826ACE70A26AF
:1073D000AAE7302CA0D0A7E7BDE8F087084B37B567
:1073E0001C68084D236A002B08BF2B4600931346E8
:1073F0000A4601462046FFF769FF03B030BD00BFD3
:10740000F00200202401002049B1FF2A85BF8A2311
:1074100003600A704FF0FF3098BF012070470846A4
:107420007047F0B506694B11B34200F1140527DA35
:1074300011F01F0105EB860605EB830201D12946F9
:1074400016E0141D55F823202B46C1F1200ECA402A
:10745000B44209D2276807FA0EF73A4343F8042BDF
:1074600054F8042BCA40F3E71A6052B1043308E021
:10747000B2420B4605D252F8043B41F8043BF7E711
:107480002B465B1B9B10036103B94361F0BDA0F168
:107490003003092B01D820380AE0A0F16103052B45
:1074A00001D8473804E0A0F14103052B02D8273862
:1074B000C0B27047002070472DE9F04F8BB00290AA
:1074C00016988A469046069300F0C9FA03684FF072
:1074D000000B18460393FFF7B5F8039B0190034494
:1074E00013F8013C0793DAF8003002331F4613F813
:1074F000010B302802D10BF1010BF7E7FFF7C7FFB3
:107500000446E0B9019A0399384601F0F9F90028D8
:1075100034D1019BF85CFE18FFF7B9FF80B3334606
:1075200018781F46302803F10103F9D0FFF7AFFFA9
:10753000B0FA80F534466D094FF0010B01E00025EB
:107540002C463A46164630780132FFF7A0FF002855
:10755000F8D1019A0399304601F0D2F950B954B9E3
:10756000019BF4182246164630780132FFF78FFF50
:107570000028F8D134B1A41BA40003E03E4600E08B
:10758000044601253378502B01D0702B2AD1737813
:107590002B2B08D02D2B03D0711C4FF0000905E0D8
:1075A0004FF0010901E04FF00009B11C0878FFF726
:1075B0006EFF431EDBB2182B14D8A0F1100211F895
:1075C000010FFFF764FF431EDBB2182B04D80A2318
:1075D00003FB0202103AF2E7B9F1000F00D0524269
:1075E000144400E03146CAF800102DB1BBF1000F81
:1075F00014BF002006207CE12946F31B013B072B2A
:1076000002DD01315B10FAE7029800F02AFA4FF030
:1076100000090546CB46019B00F1140AC3F10103A2
:10762000CDF810A00893B7422FD2731E0593079A86
:1076300016F8013C93420BD0BBF1200F16D1049BEE
:10764000C3F8009004334FF000090493CB460DE0DB
:10765000059B089A13449F42EED81846019A039955
:10766000099301F04DF9099B68B1E5E716F8010CA3
:10767000FFF70DFF00F00F0000FA0BF0059B49EA41
:1076800000090BF1040B1E46CDE7049840F8049B5B
:10769000CAEB0000801028614701484600F0A6FAB6
:1076A000D8F80060381AB04226DD871B39462846D4
:1076B00000F09DFDC8B17B1E591103F01F024FF071
:1076C00001095AF8211009FA02F20A420ED04B457C
:1076D00002DC4FF0020909E0B91E284600F087FDE0
:1076E0000028F6D04FF0030900E0814639462846CD
:1076F000FFF797FE3C440CE009DA371A29463A4670
:10770000029800F0A7FB0546E41B00F1140A4FF0B5
:107710000009D8F808309C4208DD0298294600F09C
:10772000D5F9149A00231360A320E2E0D8F80400EE
:10773000844253DA041BA6422EDCD8F80C30022B0C
:107740001AD0032B1CD0012B1DD1A6421BD1012E18
:107750000BDCD8F80430069A6220136001232B61F9
:10776000CAF80030149B1D60C3E0711E284600F06B
:107770003EFD0028EDD106E0159B002BE9D002E08C
:10778000159B002BE5D10298294600F09FF9149A29
:10779000002313605020ACE0671EB9F1000F06D142
:1077A0003FB13946284600F022FD814601E04FF006
:1077B00001097A11012307F01F0703FA07F75AF8A6
:1077C000223021461F42284618BF49F00209361BC5
:1077D000FFF727FE0227D8F8044000E00127B9F19F
:1077E000000F00F08180D8F80C30022B0ED0032B54
:1077F00010D0012B76D119F0020F73D0DAF8000007
:1078000049EA000919F0010F07D16BE0159BC3F19C
:1078100001031593159B002B64D0D5F810A005F13A
:1078200014034FEA8A0903EB090100201A68B2F138
:10783000FF3F02D001321A6020E043F8040B994266
:10784000F4D8AB689A4512DB69680298013100F000
:1078500008F983462A6905F10C01023292000C30C6
:10786000FEF790FE2946029800F030F95D462B693C
:107870005A1C2A6105EB830301225A61022F05F18C
:10788000140211D1D8F80030013B9E4227D171116A
:10789000012306F01F0603FA06F652F821301E42B5
:1078A0000CBF022701271AE02B699A450ADA012149
:1078B0002846FFF7B6FDD8F8083001349C423FF760
:1078C0002CAF0BE016F01F0608D0914459F8040CB9
:1078D00000F08CF9C6F12006B042E8DB012747F042
:1078E000200701E047F010073846149B1D60069BF7
:1078F0001C600BB0BDE8F08FC2F10802920070B5B9
:10790000C2F120064368056803FA06F42C43D3400D
:10791000046040F8043F8842F4D370BD30B503687A
:1079200011F8014B01334CB11A78A2F14105192D20
:1079300098BF2032A242F3D0002030BD0360012066
:1079400030BD0B682DE9F04F5E1102EB860613F097
:107950001F0318BF0436351F174600228246A8466B
:107960002C46914685B0D0F800B0019346F8042C1F
:1079700000921BF8011F00293CD008460392029197
:10798000FFF785FD039A00BB0299202916D8009BBA
:107990009945EEDD444505D2072A03DC41462046E1
:1079A000FFF7AAFFBC4223D90023A4F1040844F83E
:1079B000043CCDF8009044461A46DAE7292948D11C
:1079C0000BF10103CAF8003014E00132082A09F172
:1079D000010906DDBC42CCD9002344F8043C012255
:1079E000043C216800F00F0040EA01102060C0E76D
:1079F0000822BEE7B9F1000F2BD0444505D2072A73
:107A000003DC41462046FFF777FFBC420CD93B46DA
:107A100054F8042BA54243F8042BF9D2002243F872
:107A2000042B9D42FBD20BE0019B4BB1C3F1200222
:107A30004FF0FF33D34056F8042C134046F8043C73
:107A40002B6843B9BD4202D101232B6003E0043D02
:107A5000F6E7042000E0052005B0BDE8F08FF03027
:107A6000704770B5456A04460E463DB9102000F0D7
:107A70005DFF6062456085600560C560656AEB68B2
:107A800043B1636ADB6853F8260078B1026843F8B3
:107A9000262017E021220421204600F0CAFB636A59
:107AA000E860DB68002BECD1002070BD012101FAF9
:107AB00006F56A1D9200204600F0BBFB0028F3D0BB
:107AC0004660856000230361C36070BD70B5446A81
:107AD00006460D463CB9102000F028FF7062446055
:107AE00084600460C4603DB1736A6A68DB6853F8FF
:107AF0002210296043F8225070BD2DE9F04106465E
:107B00000C460D691F4601F1140E0023DEF800003B
:107B1000013381B202FB0171000C0F0C02FB0070FB
:107B200089B201EB00419D424FEA10474EF8041B19
:107B3000ECDCD7B1A3689D4212DB616830460131AD
:107B4000FFF78FFF8046226904F10C010232920098
:107B50000C30FEF717FD21463046FFF7B7FF4446CD
:107B600004EB850301355F6125612046BDE8F081A6
:107B70002DE9F843064615461F46092208330C46F0
:107B800093FBF2F3002101229A4202DA5200013102
:107B9000FAE73046FFF765FF089B092D43614FF078
:107BA0000103036111DD04F10908C1462C4419F8F1
:107BB000013B0146303B0A223046FFF79EFFA145BC
:107BC000F5D108EB0504083C01E00A3409252D1B1A
:107BD00063199F4208DD14F8013B0146303B0A223D
:107BE0003046FFF78AFFF3E7BDE8F883030C1B0478
:107BF00013B90004102300E0002310F07F4F04BFEE
:107C00000002083310F0704F04BF0001043310F07D
:107C1000404F04BF80000233002803DB420003D53D
:107C2000581C70471846704720207047036813F0AF
:107C300007020BD0D90722D49A074BBF5B089B08D9
:107C4000036003604CBF01200220704799B209B95C
:107C50001B0C102213F0FF0F04BF1B0A0832190778
:107C600004BF1B090432990704BF9B080232D907DD
:107C700002D45B0805D00132036010467047002033
:107C800070472020704710B50C460121FFF7E9FE30
:107C900001224461026110BD2DE9F74F14460A69C3
:107CA000236988469A42BEBF0B46A0461C46D8F8B8
:107CB0001070D4F81090D8F80830D8F8041007EBFA
:107CC00009069E42C8BF0131FFF7CBFE00F1140543
:107CD0002B4605EB860C0022634502D243F8042BA9
:107CE000FAE704F1140208F1140102EB890301EB35
:107CF00087070093009B0192934257D9B2F800B0D6
:107D0000BBF1000F23D08946AE464FF0000859F86A
:107D1000044BBEF800A0A3B20BFB03A34FEA144A26
:107D2000DEF8004043444FEA14480BFB0A84F24655
:107D300004EB13449BB243EA04434F454FEA144813
:107D40004AF8043B01D9D646E1E7CEF80480019B0E
:107D50000432B3F802A0BAF1000F21D02C468946B4
:107D60002B684FF00008B9F800E0B4F802B09BB2FD
:107D70000AFB0EBEA346F04443EA08434BF8043B1B
:107D800059F8043BB4F804E01B0C0AFB03E34F452D
:107D900003EB18434FEA134801D95C46E3E76360FD
:107DA0000435A7E75CF8043D13B9013E002EF9DC69
:107DB000066103B0BDE8F08F2DE9F843154612F0D7
:107DC000030206460F4607D0214C013A002354F81F
:107DD0002220FFF792FE0746AD1036D0746A3CB9F8
:107DE000102000F0A3FD7062446084600460C460F1
:107DF000D6F82480D8F808404CB940F271213046BA
:107E0000FFF741FF04460023C8F8080003604FF065
:107E10000008EB070AD5394622463046FFF73CFFFB
:107E2000814639463046FFF751FE4F466D100CD063
:107E3000206808B10446ECE7224621463046FFF7A9
:107E40002BFF2060C0F80080F4E73846BDE8F883D7
:107E5000C09F00082DE9F0470C4607469146266969
:107E60004FEA621A56444968A368751CAB4202DAAD
:107E700001315B00FAE73846FFF7F3FD0023804647
:107E80001A4600F11401534503DA41F82320013367
:107E9000F9E72AEAEA73206901EB830319F01F0965
:107EA00004F1140101EB800E14D0C9F1200C002262
:107EB00008689A4600FA09F0024343F8042B51F887
:107EC000042B8E4522FA0CF2F2D8CAF8042042B1F3
:107ED000B51C06E0043B51F8042B8E4543F8042FF3
:107EE000F9D8013D3846C8F810502146FFF7EEFD9D
:107EF0004046BDE8F08703690A6910B59B1A11D1A5
:107F000092001430143183180A4453F8044D52F887
:107F1000041D8C4202D007D3012010BD9842F4D337
:107F2000002010BD184610BD4FF0FF3010BD2DE9E8
:107F3000F8430C460746114620461546FFF7DBFF7F
:107F4000061E08D131463846FFF78BFD0123036139
:107F50004661BDE8F883BCBF23462C4638466168BD
:107F6000BABF1D4601260026FFF77BFD2B69C660C0
:107F7000266905F1140904F1140101EB860709EBE8
:107F8000830800F114054FF0000C51F8042B59F848
:107F9000044B93B29C44A3B2240CC3EB0C03C4EB7C
:107FA000124202EB23429BB24FEA224CC84543EAFD
:107FB00002428E4645F8042BE7D8BE450ED25EF845
:107FC000041B8AB26244131403EB114392B242EAD7
:107FD00003424FEA234C45F8042BEEE755F8043DE5
:107FE0000BB9013EFAE70661BDE8F883104B0B4080
:107FF000A3F15073002B02DD0020194670475B424D
:108000001B15132B4FF000004FF0000104DC4FF460
:10801000002242FA03F17047143B1E2B4FF001027D
:10802000CEBF1346C3F11F0302FA03F3184670478D
:108030000000F07FF8B5056900F1140606EB850530
:1080400055F8044C2F1F2046FFF7D0FDC0F1200348
:108050000A280B6014DCC0F10B0E24FA0EF1BE42AC
:1080600041F07F5334BF55F8081C0021153004FA45
:1080700000F021FA0EF143F4401340EA010223E03C
:10808000BE423ABFA5F1080755F8081C00210B387D
:1080900015D08440C0F1200544F07F5444F44014CE
:1080A000B74221FA05FE44EA0E038CBF57F8044C90
:1080B000002401FA00F0EC4040EA040204E00A4621
:1080C00044F07F5343F4401310461946F8BD2DE9A0
:1080D000F3411C4601219046089E099DFFF7C1FC13
:1080E000C4F31302C4F30A5407460CB142F48012DD
:1080F0000192B8F1000F19D002A840F8088DFFF7DF
:1081000095FD009B48B1019AC0F1200102FA01F1EE
:108110000B43C2407B61019200E07B61019B002B1D
:1081200014BF02210121BB61396107E001A8FFF7FB
:108130007DFD019B01217B613961203034B1A4F2C6
:10814000334404443460C0F1350009E0A0F2324009
:1081500007EB810330601869FFF748FDC0EB411061
:108160002860384602B0BDE8F0812DE9F743884623
:1081700069468146FFF75EFF0D46044601A9404669
:10818000FFF758FF0F460646D9F81030D8F81020F0
:1081900020469A1A9DE80A00C91A01EB4213002BE7
:1081A000CCBF05EB0355A7EB035732463B462946A8
:1081B000FCF7C8FD03B0BDE8F083013910B54911E3
:1081C0001469013102F1140300EB810103EB840413
:1081D000A342024604D253F8042B40F8042BF7E7DD
:1081E00000238A4202D242F8043BFAE710BD00F1B4
:1081F000140200694B11984210B50CDB0CDD11F034
:108200001F0109D052F8234024FA01F000FA01F1CD
:108210008C420CD100E0034602EB8303934204D965
:1082200053F8041D0029F9D001E0002010BD012001
:1082300010BD38B502FB01F4214600F009F80546EF
:1082400018B122460021FEF7A8F9284638BD0000E3
:1082500070B5CD1C25F0030508350C2D38BF0C2555
:10826000002D064601DBA94202D90C23336046E00B
:1082700000F08DFB234B1C681A462146A1B10B6808
:108280005B1B0ED40B2B03D90B60CC18CD501EE01A
:108290008C420BBF63684B681360636018BF0C4669
:1082A00015E00C464968E9E7174C23681BB93046CE
:1082B00000F016FB20602946304600F011FB431CFD
:1082C00018D0C41C24F00304A0420DD12560304610
:1082D00000F05EFB04F10B00231D20F00700C31A21
:1082E0000ED05A42E25070BD211A304600F0F8FA22
:1082F0000130EBD10C233360304600F049FB002005
:1083000070BD00BF2C060020280600202DE9F04794
:108310008E6882469E420C46914698463ED88A898F
:1083200012F4906F3AD02568096902236F1A6569C3
:1083300005EB450595FBF3F57B1C43449D4238BF97
:108340001D4653050FD52946FFF782FF064698B113
:108350003A462169FEF716F9A38923F4906343F0A6
:108360008003A38113E02A4600F060FB064670B943
:108370002169504600F00EFB0C23CAF80030A38997
:108380004FF0FF3043F04003A381BDE8F087266142
:108390003E44266046466561ED1BA560464528BF04
:1083A000464649463246206800F0D6FAA3680020C7
:1083B0009B1BA36023681E442660BDE8F087000075
:1083C0002DE9F04F9DB003938B8980461C060D4626
:1083D00016460DD50B695BB94021FFF739FF2860C0
:1083E000286118B90C23C8F80030CDE040236B6138
:1083F0000023099320238DF82930DFF89CB1302326
:108400008DF82A3037463C4614F8013B1BB9B7EBD0
:10841000060910D003E0252BF9D02746F3E74B4699
:10842000324629464046FFF771FF013000F0A78031
:10843000099B4B4409933B78002B00F0A08000235C
:108440004FF0FF3204930793059206938DF8533053
:108450001A930126052221784E4800F06FFA671C16
:10846000049B38B14B4A3C46801A06FA00F0184388
:108470000490EFE7D90644BF20228DF853201A0755
:1084800044BF2B228DF8532022782A2A03D0079A42
:1084900000210A200BE0039A111D12680391002AA3
:1084A00010DA524243F00200079204900BE0274694
:1084B0003B780134303B092B03D800FB0232012109
:1084C000F5E701B107923B782E2B1ED17B782A2B42
:1084D0000AD1039B02371A1D1B680392002BB8BFF9
:1084E0004FF0FF33059310E0002319460593781CE5
:1084F0000A2407463A780130303A092A03D804FBA7
:1085000001210123F5E703B10591032239782248BF
:1085100000F014FA40B14023CBEB000003FA00F066
:10852000049B013718430490397806221B487E1CAF
:108530008DF8281000F002FA88B1194B33B9039B6B
:10854000073323F007030833039314E003AB0093CE
:108550002A46144B04A94046AFF3008007E003AB62
:1085600000932A460F4B04A9404600F093F8B0F15F
:10857000FF3F824603D0099B5344099342E7AB89EE
:108580005B0601D4099801E04FF0FF301DB0BDE853
:10859000F08F00BFCC9F0008D29F0008D69F000834
:1085A000000000000D8300082DE9F04791461F46AA
:1085B0000A698B6806469342B8BF1346C9F8003073
:1085C00091F843200C46DDF8208012B10133C9F840
:1085D00000302368990642BFD9F800300233C9F849
:1085E0000030256815F0060510D104F1190A07E0DE
:1085F0000123524639463046C04701301AD0013572
:10860000E368D9F800209B1A9D42F1DB94F84330CF
:108610002268003318BF012392060FD5E1183020DD
:1086200081F843005A1C94F845102244023382F822
:10863000431003E04FF0FF30BDE8F08704F1430240
:1086400039463046C0470130F4D02268D9F800508E
:10865000E36802F00602042A08BF5D1B2269A368D2
:108660000CBF25EAE57500259342C4BF9B1AED189F
:108670004FF000091A344D4509D0012322463946EE
:108680003046C0470130D5D009F10109F3E7002099
:10869000BDE8F0872DE9F04317460A7E85B06E2AC3
:1086A000984606460C460C9B01F1430E00F0AE8046
:1086B00011D8632A22D009D8002A00F0BB80582A9A
:1086C00040F0CA8081F84520834955E0642A1ED0D5
:1086D000692A1CD0C0E0732A00F0B08009D86F2A44
:1086E0002ED0702A40F0B8800A6842F020020A605A
:1086F0003EE0752A24D0782A3AD0ADE01A6801F11C
:108700004205111D1960136884F84230A8E0216801
:108710001A6811F0800F02D0111D196008E011F0E5
:10872000400F02F10401196002D0B2F9003000E0FC
:108730001368002B3CDA2D225B4284F8432037E09B
:1087400021681A6811F0800F02D0111D196007E02E
:1087500011F0400F02F10401196001D0138800E00C
:108760001368227E5C496F2A14BF0A2208221BE08C
:1087700078225A4984F845202268186812F0800F40
:1087800000F104051D6003D1550601D5038800E002
:108790000368D00744BF42F0200222601BB9226860
:1087A00022F0200222601022002084F8430001E021
:1087B00049490A226568002DA56008DB206820F081
:1087C000040020602BB9002D7DD175460CE0002BF4
:1087D00079D07546B3FBF2F002FB1033CB5C05F8A1
:1087E000013D03460028F5D1082A0BD12368DA079A
:1087F00008D5236962689A42DEBF302305F8013C40
:1088000005F1FF35C5EB0E0323612EE008681A68F9
:1088100010F0800F496903D0101D1860136808E03C
:1088200010F0400F02F104001860136801D01980A5
:1088300000E0196000232361754616E01A68111DD7
:108840001960156800216268284600F077F808B1C1
:10885000401B6060636804E004F1420584F8422034
:1088600001232361002384F84330CDF800803B4688
:1088700003AA21463046FFF797FE013002D14FF0A0
:10888000FF3026E023692A4639463046C04701308A
:10889000F5D023689B0710D5002504F1190907E0DE
:1088A00001234A4639463046C0470130E7D00135FA
:1088B000E368039A9B1A9D42F2DBE068039B9842AF
:1088C000B8BF184605E00B7804F1420584F8423041
:1088D0008AE705B0BDE8F083DD9F0008EE9F000841
:1088E00038B5064C0023054608462360FBF7E8F937
:1088F000431C02D1236803B12B6038BD2C09002032
:1089000030B582B1451E013915F8013F11F8014F0C
:10891000A34206D1EC431444E04201D0002BF3D132
:108920001C46181B30BD104630BD0000024B0146EE
:108930001868FFF78DBC00BFF002002010B5C9B267
:1089400002449042034605D01C7801308C42F8D195
:10895000184610BD002010BD884210B501EB02037F
:1089600001D8421E0BE09842FBD28118D21AD342A2
:1089700004D013F8014D01F8014DF8E710BD9942FC
:1089800004D011F8014B02F8014FF8E710BD704711
:108990007047000038B50546002944D051F8043C22
:1089A0000C1F002BB8BFE418FFF7F1FF1E4A136835
:1089B000114613B96360146030E0A3420DD92268F8
:1089C000A018834201BF18685B68121822606360B8
:1089D0000C6023E0A24203D813465A68002AF9D15A
:1089E00018681918A1420BD1216801445818824215
:1089F000196013D110685268014419605A600DE083
:108A000002D90C232B6009E021686018824201BF63
:108A1000106852680918216062605C602846BDE8F1
:108A20003840FFF7B5BF38BD2C060020F8B5074623
:108A300015460E4621B91146BDE8F840FFF708BCBF
:108A40001AB9FFF7A7FF2846F8BD00F015F88542D0
:108A50000ED929463846FFF7FBFB044650B1314694
:108A60002A46FDF78FFD31463846FFF793FF01E0B8
:108A70003046F8BD2046F8BD51F8040C0028BEBFB2
:108A8000091851F8043CC018043870474FF0FF3CF7
:108A900006E000BF4FF0010C02E000BF4FF0010CF8
:108AA0004DF804CD4FEA410C7FEA6C5C4FEA430C71
:108AB00018BF7FEA6C5C1BD001B050EA410C0CBFC0
:108AC00052EA430C91EA030F02BF90EA020F002022
:108AD000704710F1000F91EA030F58BF994208BF89
:108AE00090422CBFD8176FEAE37040F00100704746
:108AF0004FEA410C7FEA6C5C02D150EA013C07D19D
:108B00004FEA430C7FEA6C5CD6D152EA033CD3D0E7
:108B10005DF8040B704700BF8446104662468C46E1
:108B20001946634600E000BF01B5FFF7B7FF002814
:108B300048BF10F1000F01BD4DF808EDFFF7F4FF3D
:108B40000CBF012000205DF808FB00BF4DF808EDC8
:108B5000FFF7EAFF34BF012000205DF808FB00BFEB
:108B60004DF808EDFFF7E0FF94BF012000205DF80D
:108B700008FB00BF4DF808EDFFF7CEFF94BF0120C2
:108B800000205DF808FB00BF4DF808EDFFF7C4FFBB
:108B900034BF012000205DF808FB00BF4A0011D25D
:108BA00012F5001211D20DD56FF47873B3EB625247
:108BB0000ED44FEAC12343F0004343EA505323FA53
:108BC00002F070474FF00000704750EA013002D1C8
:108BD0004FF0FF3070474FF000007047C49B000813
:108BE000C89B0008CC9B0008D09B0008D49B0008C1
:108BF000DC9B0008E09B0008E49B00084F4B0A0D3B
:108C0000636D643E000000004F4600004F4E206F31
:108C100072204F464620616C6C6F776564206F6EE2
:108C20006C790A0D636D643E000000004F4E0A0D22
:108C3000000000004F46460A0D00000048454C5019
:108C4000000000003F0000000A0D416C6C6F77656A
:108C50006420636F6D6D616E647320286E6F742085
:108C6000636173652073656E736974697665293A0B
:108C70000A0D0A0D00000000425554544F4E206F5B
:108C80006E2F6F6666202D20757365206275747473
:108C90006F6E20746F207475726E206F66660A0D99
:108CA000000000004C454453206F6E2F6F66662015
:108CB0002D20757365204C4544730A0D000000009B
:108CC000504F574552206E202D20726620706F77CE
:108CD0006572206E203D203020746F2037202837A9
:108CE000206973206D61782E290A0D00484F4C448D
:108CF0004F4646206E202D206E203D2074696D6504
:108D0000206265747765656E2074776F2072747465
:108D100079206D6573736167657320696E20736573
:108D2000636F6E64730A0D00534552434F4D206EBE
:108D3000202D207370656564206F662073657269ED
:108D4000616C20636F6D6D756E69636174696F6EC0
:108D500020706F727420286E203D203330302074D4
:108D60006F20313135323030290A0D0052545459B8
:108D7000206F6E2F6F6666202D2073656E642072E3
:108D8000747479206D6573736167650A0D00000066
:108D900052545459465251206E2E6E202D206E2E64
:108DA0006E203D207274747920616E64206377694F
:108DB00064206672657175656E637920696E204DF9
:108DC000487A0A0D000000005254545943414C4C5B
:108DD00020737472696E67202D2072747479206319
:108DE000616C6C7369676E2028757020746F203118
:108DF000352063686172616374657273290A0D00BE
:108E000042415544206E202D206E203D2072747406
:108E10007920626175647261746520286D61782EB5
:108E200020333030290A0D004442495453206E202B
:108E30002D206E203D20727474792064617461620B
:108E4000697473202837206F722038290A0D0000BA
:108E50005342495453206E202D206E203D207274C1
:108E600074792073746F70206269747320283120C4
:108E70006F722032290A0D005348494654206E2053
:108E80002D206E203D20312C322C332C34206F725B
:108E9000203237302C3534302C3831302C313038CA
:108EA0003020487A0A0D000054454D5020286F723A
:108EB0002054454D504552415455524529206F6E1E
:108EC0002F6F6666202D2073656E642074656D704B
:108ED0006572617475726520696E20727474792090
:108EE0006D657373616765730A0D0000414C542012
:108EF000286F7220414C54495455444529206F6EC7
:108F00002F6F6666202D2073656E6420616C746916
:108F10007475646520696E2072747479206D657350
:108F200073616765730A0D005350454544206F6EA9
:108F30002F6F6666202D2073656E642073706565E3
:108F40006420696E2072747479206D657373616733
:108F500065730A0D00000000434F55525345206FC2
:108F60006E2F6F6666202D2073656E6420636F75AB
:108F700072736520696E2072747479206D657373E5
:108F8000616765730A0D000055424154206F6E2FD2
:108F90006F6666202D2073656E642062617474654F
:108FA000727920766F6C7461676520696E207274C7
:108FB0007479206D657373616765730A0D00000035
:108FC000525454595F57574C206E202D206E203D2F
:108FD0002063686172616374657273206F662077C5
:108FE000776C6F6361746F7220286F6E6C79206587
:108FF00076656E206E756D626572732920696E20CC
:1090000072747479206D657373616765730A0D00FE
:10901000525454595F54494D45206F6E2F6F666608
:10902000202D2073656E642074696D6520696E2043
:1090300072747479206D657373616765730A0D00CE
:1090400053415420286F7220534154454C4C49548D
:10905000455329206F6E2F6F6666202D2073656E35
:109060006420686561726420736174656C6C6974F6
:10907000657320696E2072747479206D65737361F5
:109080006765730A0D00000041505253206F6E2F28
:109090006F6666202D2073656E6420617072732088
:1090A0006D657373616765730A0D0000415052531B
:1090B000465251206E2E6E202D206E2E6E203D20A9
:1090C00061707273206672657175656E637920696F
:1090D0006E204D487A0A0D004150525343414C4C8A
:1090E00020737472696E67202D2061707273206323
:1090F000616C6C7369676E2028757020746F203600
:109100002063686172616374657273290A0D0000DF
:1091100053534944206E202D206170727320737365
:109120006964206E203D203120746F2031350A0D96
:1091300000000000415052535F414C54206F6E2F8D
:109140006F6666202D2073656E6420616C7469748F
:1091500075646520696E206170727320747465781F
:10916000740A0D0053594D424F4C20737472696E4E
:1091700067202D2073796D626F6C2066726F6D2091
:10918000617072732073796D626F6C207461626CB0
:109190006520283220636861726163746572732987
:1091A0000A0D000052454C415920737472696E6774
:1091B000202D20617072732072656C617973202894
:1091C00057494445312D312C57494445322D3129D9
:1091D0000A0D0000415052535F4556455259206ECA
:1091E000202D2074696D65206265747765656E2039
:1091F00061707273206D6573736167657320697345
:10920000206E207820686F6C646F66660A0D00001F
:109210005441494C5F4556455259206E202D2074CB
:10922000696D65206265747765656E207461696C2F
:109230002074657874206973206E207820617072C4
:10924000732074696D652C2030203D206E6F207472
:1092500061696C20746578740A0D00005454455897
:109260005420737472696E67202D207461696C20BC
:10927000746578742028757020746F203130302028
:1092800063686172616374657273290A0D0000007E
:10929000415052535F55424154206F6E2F6F6666A6
:1092A000202D2073656E642062617474657279206C
:1092B000766F6C7461676520696E206170727320CF
:1092C00074746578740A0D00415052535F54454DD3
:1092D00050206F6E2F6F6666202D2073656E6420A0
:1092E000726164696F20636869702074656D706570
:1092F00072617475726520696E206170727320747A
:10930000746578740A0D000043574944206F6E2F2E
:109310006F6666202D2073656E6420637769642014
:109320006D657373616765730A0D000043574944A7
:109330004D45535320737472696E67202D206377F7
:10934000206D6573736167652028757020746F20C8
:1093500032352063686172616374657273290A0D26
:1093600000000000435749445F414C54206F6E2F6A
:109370006F6666202D2073656E6420616C7469745D
:10938000756465207669612063770A0D000000002E
:10939000435749445F55424154206F6E2F6F6666B4
:1093A000202D2073656E642062617474657279206B
:1093B000766F6C74616765207669612063770A0D4A
:1093C00000000000435749445F57574C206E202D42
:1093D000206E203D20636861726163746572732042
:1093E0006F662077776C6F6361746F7220286F6E81
:1093F0006C79206576656E206E756D626572732975
:1094000020696E204357206D657373616765730A29
:109410000D000000435749445F4556455259206EA0
:10942000202D2074696D65206265747765656E20F6
:109430006377206D65737361676573206973206E50
:10944000207820686F6C646F66660A0D000000006B
:1094500043575F5350454544206E206E203D2063A6
:109460007720737065656420696E2077706D0A0DD2
:109470000000000044495350202D2073686F77206E
:10948000706172616D65746572730A0D0000000091
:10949000444546202D207365742064656661756CB3
:1094A000742076616C7565730A0D00005341564552
:1094B000202D207361766520706172616D65746521
:1094C000727320746F20666C6173680A0D0000006F
:1094D00044495350000000000A0D43757272656ED6
:1094E0007420706172616D65746572733A0A0D0A59
:1094F00000000000425554544F4E20004C45445348
:1095000020000000504F57455220617070726F78F4
:109510002E202573206D570A0D000000554152542E
:1095200020256420382D4E2D310A0D00484F4C4423
:109530004F464620256C6420730A0D00525454593E
:10954000200000005254545920616E642043574952
:1095500044204652455155454E43593A20253364DF
:109560002E25303364204D487A0A0D005254545948
:109570002043414C4C5349474E3A2025730A0D0075
:10958000525454592042415544524154453A2025A1
:10959000642042640A0D0000525454592053484933
:1095A00046543A20256420487A0A0D0052545459F2
:1095B000204441544120424954533A2025640A0D25
:1095C00000000000525454592053544F5020424937
:1095D00054533A2025640A0D000000005254545997
:1095E0002054454D50455241545552453A200000B3
:1095F0005254545920414C5449545544453A200042
:10960000525454592053504545443A20000000001C
:109610005254545920434F555253453A20000000AC
:1096200052545459204241545445525920564F4C9B
:10963000544147453A200000525454592053415454
:10964000454C4C495445533A20000000525454595B
:109650002057574C3A202564206368617261637417
:109660006572730A0D000000525454592057574C2C
:109670003A204F46460A0D00525454592054494D41
:10968000453A2000415052532000000041505253AF
:10969000204652455155454E43593A202533642EB4
:1096A00025303364204D487A0A0D00004150525352
:1096B0002043414C4C5349474E3A2025732D256495
:1096C0000A0D0000415052532052454C41593A2056
:1096D00025730A0D00000000415052532053594D8C
:1096E000424F4C3A2025730A0D000000415052535E
:1096F0002045564552593A2025640A0D00000000C5
:109700004150525320414C543A2000004150525392
:10971000205441494C2054455854204556455259EF
:109720003A2025640A0D000041505253205441490B
:109730004C20544558543A2025730A0D000000006F
:109740004150525320554241543A20004150525307
:109750002054454D503A2000435749442000000012
:1097600043574944204D4553534147453A20000053
:109770000A0D435749442053504545443A20256437
:109780002057504D0A0D0000435749442045564587
:1097900052593A2025640A0D0000000043574944FD
:1097A0002057574C3A2025642063686172616374C6
:1097B0006572730A0D000000435749442057574C07
:1097C0003A204F46460A0D0043574944205542412E
:1097D000543A20004357494420414C543A20000059
:1097E0005454455854000000546F6F206D616E79D9
:1097F00020636861726163746572730A0D636D64DE
:109800003E0000005254545943414C4C00000000AB
:109810004150525343414C4C000000004F6E6C7954
:10982000206C65747465727320616E64206E756D52
:10983000626572732061726520616C6C6F7765641C
:109840000A0D636D643E0000435749444D45535330
:109850000000000052454C4159000000504F574550
:1098600052000000506F77657220617070726F78DF
:109870002E202573206D570A0D636D643E00000095
:109880003020746F203720616C6C6F776564206FB7
:109890006E6C790A0D636D643E00000043574944C5
:1098A0005F57574C000000003020746F2031322089
:1098B000616C6C6F776564206F6E6C790A0D636DF7
:1098C000643E0000525454595F57574C000000004A
:1098D0004241554400000000323520746F2033307F
:1098E0003020616C6C6F776564206F6E6C790A0D47
:1098F000636D643E000000004150525346525100D7
:109900004672657175656E6379206F7574206F6638
:109910002072616E6765203234302E302D3933303D
:109920002E30204D487A0A0D636D643E0000000021
:109930005254545946525100484F4C444F464600E9
:10994000444249545300000037206F722038206190
:109950006C6C6F776564206F6E6C790A0D636D6453
:109960003E000000534249545300000031206F7202
:10997000203220616C6C6F776564206F6E6C790AA1
:109980000D636D643E0000005348494654000000DA
:10999000312C322C332C34206F72203237302C355E
:1099A00034302C3831302C3130383020616C6C6FD1
:1099B000776564206F6E6C790A0D636D643E0000FC
:1099C00053534944000000006F6E6C792066726F3B
:1099D0006D203020746F2031350A0D636D643E00B8
:1099E000534552434F4D000033303020746F2031C7
:1099F000313532303020616C6C6F776564206F6E6A
:109A00006C790A0D636D643E0000000053594D42AD
:109A10004F4C000043686172616374657273206922
:109A200073206E6F742076616C69640A0D636D64D7
:109A30003E000000425554544F4E00004C454453E4
:109A4000000000005254545900000000415052538D
:109A5000000000004357494400000000525454598C
:109A60005F54494D45000000435749445F414C5401
:109A700000000000435749445F5542415400000034
:109A800054454D500000000054454D50455245543A
:109A9000555245005350454544000000434F555230
:109AA00053450000414C5400414C544954554445E1
:109AB0000000000055424154000000004150525344
:109AC0005F55424154000000415052535F54454D90
:109AD0005000000053415400534154454C4C4954EC
:109AE00045530000415052535F414C540000000068
:109AF000415052535F455645525900005441494C1C
:109B00005F4556455259000043575F535045454401
:109B100000000000435749445F4556455259000034
:109B200043575F45564552590000000044454600E2
:109B3000204D6F6469666965642052532D3431206D
:109B400062616C6C6F6F6E20747261636B65720022
:109B50004E4F43414C4C0000544553542044452043
:109B60004E4F43414C4C2F414D0000002F4F000001
:109B700057494445312D31005341564500000000FE
:109B8000506172616D65746572732073617665648E
:109B9000204F4B0A0D636D643E00000043616E6E02
:109BA0006F74207361766520706172616D65746594
:109BB00072730A0D636D643E000000003F0A0D637E
:109BC0006D643E00302E3800312E3600332E3200C8
:109BD000362E330031322E360000000032350000C0
:109BE00035300000313030002D00000024242424C2
:109BF00025732C25640000002C253032753A253061
:109C000032753A25303275002C257325752E253096
:109C1000346C752C257325752E2530346C75000039
:109C20002C256C64000000002C2573002C2564009A
:109C30002C25642E25303264000000002A253034A3
:109C4000580A000020494E20257300002041534C43
:109C500020256C6400000000204241542025642E21
:109C60002530326400000000202B00000A0D4D6FEB
:109C7000646966696564205253343120666F7220CE
:109C800043572C20525454592026204150525320DF
:109C9000762E332E32206279204F4D3342430A0D07
:109CA000636D643E00000000415042435253000087
:109CB0003A5445535431323334353637383930001D
:109CC000257320416C743D256C646D00257320550F
:109CD0006261743D25642E25303264560000000018
:109CE00025732074656D703D256443002125303255
:109CF00064253032642E2530327525632F253033AC
:109D000064253032752E2530327525632563256331
:109D1000413D2530366C642F50256453256454250D
:109D200064562564202573002A73616A293F3E3CEE
:109D30003830202123272F47550131354C0106119A
:109D4000150902140B10041E0D1207050F161B0A2D
:109D500008030C180E191D13120A180A180A00001D
:109D60008096184B4300504F534958002E00000076
:109D7000BC89D897B2D29C3C33A7A8D523F64939E1
:109D80003DA7F444FD0FA5329D978CCF08BA5B2503
:109D9000436FAC642806681135000000CEFBFFFF5E
:109DA000CB03000001000000000000006E660069A7
:109DB0006E69747900616E0034000000CEFBFFFF15
:109DC000CB03000001000000000000000020202064
:109DD000202020202020282828282820202020205B
:109DE000202020202020202020202020208810102B
:109DF0001010101010101010101010101004040487
:109E00000404040404040410101010101010414144
:109E10004141414101010101010101010101010132
:109E20000101010101010101101010101010424246
:109E30004242424202020202020202020202020202
:109E400002020202020202021010101020000000A2
:109E50000000000000000000000000000000000002
:109E600000000000000000000000000000000000F2
:109E700000000000000000000000000000000000E2
:109E800000000000000000000000000000000000D2
:109E900000000000000000000000000000000000C2
:109EA00000000000000000000000000000000000B2
:109EB00000000000000000000000000000000000A2
:109EC0000000000000000000000000000000000092
:109ED000000000000000F03F0000000000002440EF
:109EE00000000000000059400000000000408F40CA
:109EF000000000000088C34000000000006AF84035
:109F00000000000080842E4100000000D012634158
:109F10000000000084D797410000000065CDCD41CE
:109F2000000000205FA00242000000E876483742AF
:109F3000000000A2941A6D42000040E59C30A2424D
:109F40000000901EC4BCD64200003426F56B0C43C2
:109F50000080E03779C3414300A0D8855734764369
:109F600000C84E676DC1AB43003D9160E458E143CA
:109F7000408CB5781DAF154450EFE2D6E41A4B443F
:109F800092D54D06CFF08044F64AE1C7022DB54484
:109F9000B49DD9794378EA440080E03779C34143DE
:109FA000176E05B5B5B89346F5F93FE9034F384D3F
:109FB000321D30F94877825A3CBF737FDD4F1575EB
:109FC00005000000190000007D000000232D302B4B
:109FD0002000686C4C0065666745464700303132AA
:109FE0003334353637383941424344454600303101
:0F9FF00032333435363738396162636465660061
:10A0000008B10181B0B000840000000008B10181F6
:08A01000B0B000840000000064
:10A018003892FF7FB0A904806492FF7F010000009E
:10A028007492FF7F03AF34806895FF7F01000000C2
:10A03800E8A1FF7FAD08B180B0A2FF7FB0B0A880D3
:10A04800F8A2FF7FB0B0AA8020A3FF7FA908B18043
:10A058004CA3FF7F01000000E0A3FF7FB0B0AE80FB
:10A068005CA4FF7F0100000080A4FF7FB0B0A8803F
:10A07800A8A4FF7FA908B180D4A4FF7FB0B0AA80AC
:10A08800F4A4FF7F01000000B4A5FF7FB0A90480FD
:10A09800E0A5FF7F0100000034B6FF7FB0A9028071
:10A0A800D0B6FF7FB0B0A88020B7FF7F01000000C6
:10A0B8002CB7FF7FB0B0AA8064B7FF7FAE71B280C3
:10A0C80030B8FF7F010000002CB8FF7FAB3F38801D
:10A0D80084B8FF7F0100000090B8FF7FB0B0AA806D
:10A0E800CCB8FF7F0100000084B9FF7FAB0EB280BF
:10A0F800ECB9FF7FB0AF0A80C0BCFF7F0100000051
:10A10800C4BCFF7FAB3F04800CBFFF7F0100000091
:10A11800E8C0FF7F00840480FCC0FF7F01000000CE
:10A12800F8C0FF7FB0AD048094C3FF7FB0A8038060
:10A13800B4C3FF7FC4FEFF7FB8C3FF7FC8FEFF7FA5
:08A14800C4C3FF7F0100000009
:10A150000100000001010100983A000064000000C5
:10A1600002070200000001010001010001010000DE
:10A170000100014D6F6469666965642052532D3496
:10A18000312062616C6C6F6F6E20747261636B65FD
:10A19000720000000000000000000000000000004D
:10A1A00000000000000000000000000000000000AF
:10A1B000000000000000000000000000000000009F
:10A1C000000000000000000000000000000000008F
:10A1D000000000000000000000013C0100004E4FA4
:10A1E00043414C4C000000004E4F43414C4C2F412A
:10A1F0004D00000000000000544553542044452009
:10A200004E4F43414C4C2F414D00000000000000D8
:10A210000000000000002F4F0000000B0040D8435A
:10A220000040D94303000000600000001900000056
:10A2300057494445312D3100000000000000000066
:10A24000000000000000000000000000000000000E
:10A25000D00700000A0000000100AB124E006400AD
:10A2600000000000010203040102030406070809BC
:10A270000204060843000000000000000000000087
:10A2800000000000000000000000000000000000CE
:10A29000000000004300000000000000000000007B
:10A2A00000000000000000000000000000000000AE
:10A2B000000000004300000000000000000000005B
:10A2C000000000000000000000000000000000008E
:10A2D000000000004300000000000000000000003B
:10A2E000000000000000000000000000000000006E
:10A2F000000000004300000000000000000000001B
:10A30000000000000000000000000000000000004D
:10A3100000000000430000000000000000000000FA
:10A32000000000000000000000000000000000002D
:10A3300000000000430000000000000000000000DA
:10A34000000000000000000000000000000000000D
:10A3500000000000097400086165000800000000AA
:10A36000CC9D00086C9D0008D19F0008D19F00087B
:10A37000D19F0008D19F0008D19F0008D19F0008FD
:10A38000D19F0008D19F0008D19F0008FFFFFFFF69
:10A39000FFFFFFFFFFFFFFFFFFFF00000100415332
:10A3A00043494900000000000000000000000000D8
:10A3B0000000000000000000000000000000415309
:10A3C00043494900000000000000000000000000B8
:10A3D000000000000000000000000000000000007D
:10A3E000000000000000000000000000000000006D
:10A3F000000000000000000000000000000000005D
:10A40000000000000000000000000000000000004C
:10A41000000000000000000000000000000000003C
:10A42000000000000000000000000000000000002C
:10A43000000000000000000000000000000000001C
:04A440009002002066
:0400000508000000EF
:00000001FF
